CCP.DAS = disassemblierter CCP		19.6.86
			ORG	0C400H
		X0000	EQU	00000H		.
		Y0003	EQU	00003H		.
		Y0004	EQU	00004H		.
		X0005	EQU	00005H		.
		Y0080	EQU	00080H		.
		X0100	EQU	00100H		.
		Y2420	EQU	02420H		.
		Y3020	EQU	03020H		.
		Y322D	EQU	0322DH		.
		Y3832	EQU	03832H		.
		XDA06	EQU	0DA06H		.
		XDA09	EQU	0DA09H		.
		XDA0C	EQU	0DA0CH		.
		XDA0F	EQU	0DA0FH		.
		XDA15	EQU	0DA15H		.
		XDA18	EQU	0DA18H		.
		XDA1B	EQU	0DA1BH		.
		XDA1E	EQU	0DA1EH		.
		XDA21	EQU	0DA21H		.
		XDA24	EQU	0DA24H		.
		XDA27	EQU	0DA27H		.
		XDA2A	EQU	0DA2AH		.
		XDA30	EQU	0DA30H		.
		XDA6E	EQU	0DA6EH		.
		XEDCE	EQU	0EDCEH		.
		XF450	EQU	0F450H		.
		XF5AB	EQU	0F5ABH		.
		XF5D8	EQU	0F5D8H		.
C400  C35CC7	DC400:	JP	AC75C		.\.
		;
		; >> NO EXECUTION PATH TO HERE <<
C403  C358C7		JP	AC758		.X.
		;
		; >> NO EXECUTION PATH TO HERE <<
M.                COPYRIGHT (C) 1979, DIGITAL RESEARCH  SERIAL NUMBER: 02-200-2283
C458  00	AC458:	NOP			.
...
C487  00	AC487:	NOP			.
C488  08	DC488:	EX	AF,AF'		.
C489  C40000		CALL	NZ,X0000	...
C48C  5F	AC48C:	LD	E,A		_
C48D  0E02		LD	C,002H		..
C48F  C30500		JP	X0005		...
		;
C492  C5	AC492:	PUSH	BC		.
C493  CD8CC4		CALL	AC48C		...
C496  C1		POP	BC		.
C497  C9		RET			.
		;
C498  3E0D	AC498:	LD	A,00DH		>.
C49A  CD92C4		CALL	AC492		...
C49D  3E0A		LD	A,00AH		>.
C49F  C392C4		JP	AC492		...
		;
C4A2  3E20	AC4A2:	LD	A,020H		> 
C4A4  C392C4		JP	AC492		...
		;
C4A7  C5	AC4A7:	PUSH	BC		.
C4A8  CD98C4		CALL	AC498		...
C4AB  E1		POP	HL		.
C4AC  7E	AC4AC:	LD	A,(HL)		~
C4AD  B7		OR	A		.
C4AE  C8		RET	Z		.
C4AF  23		INC	HL		#
C4B0  E5		PUSH	HL		.
C4B1  CD8CC4		CALL	AC48C		...
C4B4  E1		POP	HL		.
C4B5  C3ACC4		JP	AC4AC		...
		;
C4B8  0E0D	AC4B8:	LD	C,00DH		..
C4BA  C30500		JP	X0005		...
		;
C4BD  5F	AC4BD:	LD	E,A		_
C4BE  0E0E		LD	C,00EH		..
C4C0  C30500		JP	X0005		...
		;
C4C3  CD0500	AC4C3:	CALL	X0005		...
C4C6  32EECB		LD	(DCBEE),A	2..
C4C9  3C		INC	A		<
C4CA  C9		RET			.
		;
C4CB  0E0F	AC4CB:	LD	C,00FH		..
C4CD  C3C3C4		JP	AC4C3		...
		;
C4D0  AF	AC4D0:	XOR	A		.
C4D1  32EDCB		LD	(DCBED),A	2..
C4D4  11CDCB		LD	DE,DCBCD	...
C4D7  C3CBC4		JP	AC4CB		...
		;
C4DA  0E10	AC4DA:	LD	C,010H		..
C4DC  C3C3C4		JP	AC4C3		...
		;
C4DF  0E11	AC4DF:	LD	C,011H		..
C4E1  C3C3C4		JP	AC4C3		...
		;
C4E4  0E12	AC4E4:	LD	C,012H		..
C4E6  C3C3C4		JP	AC4C3		...
		;
C4E9  11CDCB	AC4E9:	LD	DE,DCBCD	...
C4EC  C3DFC4		JP	AC4DF		...
		;
C4EF  0E13	AC4EF:	LD	C,013H		..
C4F1  C30500		JP	X0005		...
		;
C4F4  CD0500	AC4F4:	CALL	X0005		...
C4F7  B7		OR	A		.
C4F8  C9		RET			.
		;
C4F9  0E14	AC4F9:	LD	C,014H		..
C4FB  C3F4C4		JP	AC4F4		...
		;
C4FE  11CDCB	AC4FE:	LD	DE,DCBCD	...
C501  C3F9C4		JP	AC4F9		...
		;
C504  0E15	AC504:	LD	C,015H		..
C506  C3F4C4		JP	AC4F4		...
		;
C509  0E16	AC509:	LD	C,016H		..
C50B  C3C3C4		JP	AC4C3		...
		;
C50E  0E17	AC50E:	LD	C,017H		..
C510  C30500		JP	X0005		...
		;
C513  1EFF	AC513:	LD	E,0FFH		..
C515  0E20	AC515:	LD	C,020H		. 
C517  C30500		JP	X0005		...
		;
C51A  CD13C5	AC51A:	CALL	AC513		...
C51D  87	AC51D:	ADD	A,A		.
C51E  87		ADD	A,A		.
C51F  87		ADD	A,A		.
C520  87		ADD	A,A		.
C521  21EFCB		LD	HL,DCBEF	!..
C524  B6		OR	(HL)		.
C525  320400		LD	(Y0004),A	2..
C528  C9		RET			.
		;
C529  3AEFCB	AC529:	LD	A,(DCBEF)	:..
C52C  320400		LD	(Y0004),A	2..
C52F  C9		RET			.
		;
C530  FE61	AC530:	CP	061H		.a
C532  D8		RET	C		.
C533  FE7B		CP	07BH		.{
C535  D0		RET	NC		.
C536  E65F		AND	05FH		._
C538  C9		RET			.
		;
C539  3AABCB	AC539:	LD	A,(DCBAB)	:..
C53C  B7		OR	A		.
C53D  CA96C5		JP	Z,AC596		...
C540  3AEFCB		LD	A,(DCBEF)	:..
C543  B7		OR	A		.
C544  3E00		LD	A,000H		>.
C546  C4BDC4		CALL	NZ,AC4BD	...
C549  11ACCB		LD	DE,TCBAC	...
C54C  CDCBC4		CALL	AC4CB		...
C54F  CA96C5		JP	Z,AC596		...
C552  3ABBCB		LD	A,(DCBBB)	:..
C555  3D		DEC	A		=
C556  32CCCB		LD	(DCBCC),A	2..
C559  11ACCB		LD	DE,TCBAC	...
C55C  CDF9C4		CALL	AC4F9		...
C55F  C296C5		JP	NZ,AC596	...
C562  1107C4		LD	DE,AC407	...
C565  218000		LD	HL,00080H	!..
C568  0680		LD	B,080H		..
C56A  CD42C8		CALL	AC842		.B.
C56D  21BACB		LD	HL,TCBBA	!..
C570  3600		LD	(HL),000H	6.
C572  23		INC	HL		#
C573  35		DEC	(HL)		5
C574  11ACCB		LD	DE,TCBAC	...
C577  CDDAC4		CALL	AC4DA		...
C57A  CA96C5		JP	Z,AC596		...
C57D  3AEFCB		LD	A,(DCBEF)	:..
C580  B7		OR	A		.
C581  C4BDC4		CALL	NZ,AC4BD	...
C584  2108C4		LD	HL,TC408	!..
C587  CDACC4		CALL	AC4AC		...
C58A  CDC2C5		CALL	AC5C2		...
C58D  CAA7C5		JP	Z,AC5A7		...
C590  CDDDC5		CALL	AC5DD		...
C593  C382C7		JP	AC782		...
		;
C596  CDDDC5	AC596:	CALL	AC5DD		...
C599  CD1AC5		CALL	AC51A		...
C59C  0E0A		LD	C,00AH		..
C59E  1106C4		LD	DE,TC406	...
C5A1  CD0500		CALL	X0005		...
C5A4  CD29C5		CALL	AC529		.).
C5A7  2107C4	AC5A7:	LD	HL,AC407	!..
C5AA  46		LD	B,(HL)		F
C5AB  23	AC5AB:	INC	HL		#
C5AC  78		LD	A,B		x
C5AD  B7		OR	A		.
C5AE  CABAC5		JP	Z,AC5BA		...
C5B1  7E		LD	A,(HL)		~
C5B2  CD30C5		CALL	AC530		.0.
C5B5  77		LD	(HL),A		w
C5B6  05		DEC	B		.
C5B7  C3ABC5		JP	AC5AB		...
		;
C5BA  77	AC5BA:	LD	(HL),A		w
C5BB  2108C4		LD	HL,TC408	!..
C5BE  2288C4		LD	(DC488),HL	"..
C5C1  C9		RET			.
		;
C5C2  0E0B	AC5C2:	LD	C,00BH		..
C5C4  CD0500		CALL	X0005		...
C5C7  B7		OR	A		.
C5C8  C8		RET	Z		.
C5C9  0E01		LD	C,001H		..
C5CB  CD0500		CALL	X0005		...
C5CE  B7		OR	A		.
C5CF  C9		RET			.
		;
C5D0  0E19	AC5D0:	LD	C,019H		..
C5D2  C30500		JP	X0005		...
		;
C5D5  118000	AC5D5:	LD	DE,00080H	...
C5D8  0E1A	AC5D8:	LD	C,01AH		..
C5DA  C30500		JP	X0005		...
		;
C5DD  21ABCB	AC5DD:	LD	HL,DCBAB	!..
C5E0  7E		LD	A,(HL)		~
C5E1  B7		OR	A		.
C5E2  C8		RET	Z		.
C5E3  3600		LD	(HL),000H	6.
C5E5  AF		XOR	A		.
C5E6  CDBDC4		CALL	AC4BD		...
C5E9  11ACCB		LD	DE,TCBAC	...
C5EC  CDEFC4		CALL	AC4EF		...
C5EF  3AEFCB		LD	A,(DCBEF)	:..
C5F2  C3BDC4		JP	AC4BD		...
		;
C5F5  1128C7	AC5F5:	LD	DE,TC728	.(.
C5F8  2100CC		LD	HL,TCC00	!..
C5FB  0606		LD	B,006H		..
C5FD  1A	AC5FD:	LD	A,(DE)		.
C5FE  BE		CP	(HL)		.
C5FF  C2CFC7		JP	NZ,AC7CF	...
C602  13		INC	DE		.
C603  23		INC	HL		#
C604  05		DEC	B		.
C605  C2FDC5		JP	NZ,AC5FD	...
C608  C9		RET			.
		;
C609  CD98C4	AC609:	CALL	AC498		...
C60C  2A8AC4		LD	HL,(DC48A)	*..
C60F  7E	AC60F:	LD	A,(HL)		~
C610  FE20		CP	020H		. 
C612  CA22C6		JP	Z,AC622		.".
C615  B7		OR	A		.
C616  CA22C6		JP	Z,AC622		.".
C619  E5		PUSH	HL		.
C61A  CD8CC4		CALL	AC48C		...
C61D  E1		POP	HL		.
C61E  23		INC	HL		#
C61F  C30FC6		JP	AC60F		...
		;
C622  3E3F	AC622:	LD	A,03FH		>?
C624  CD8CC4		CALL	AC48C		...
C627  CD98C4		CALL	AC498		...
C62A  CDDDC5		CALL	AC5DD		...
C62D  C382C7		JP	AC782		...
		;
C630  1A	AC630:	LD	A,(DE)		.
C631  B7		OR	A		.
C632  C8		RET	Z		.
C633  FE20		CP	020H		. 
C635  DA09C6		JP	C,AC609		...
C638  C8		RET	Z		.
C639  FE3D		CP	03DH		.=
C63B  C8		RET	Z		.
C63C  FE5F		CP	05FH		._
C63E  C8		RET	Z		.
C63F  FE2E		CP	02EH		..
C641  C8		RET	Z		.
C642  FE3A		CP	03AH		.:
C644  C8		RET	Z		.
C645  FE3B		CP	03BH		.;
C647  C8		RET	Z		.
C648  FE3C		CP	03CH		.<
C64A  C8		RET	Z		.
C64B  FE3E		CP	03EH		.>
C64D  C8		RET	Z		.
C64E  C9		RET			.
		;
C64F  1A	AC64F:	LD	A,(DE)		.
C650  B7		OR	A		.
C651  C8		RET	Z		.
C652  FE20		CP	020H		. 
C654  C0		RET	NZ		.
C655  13		INC	DE		.
C656  C34FC6		JP	AC64F		.O.
		;
C659  85	AC659:	ADD	A,L		.
C65A  6F		LD	L,A		o
C65B  D0		RET	NC		.
C65C  24		INC	H		$
C65D  C9		RET			.
		;
C65E  3E00	AC65E:	LD	A,000H		>.
C660  21CDCB	AC660:	LD	HL,DCBCD	!..
C663  CD59C6		CALL	AC659		.Y.
C666  E5		PUSH	HL		.
C667  E5		PUSH	HL		.
C668  AF		XOR	A		.
C669  32F0CB		LD	(DCBF0),A	2..
C66C  2A88C4		LD	HL,(DC488)	*..
C66F  EB		EX	DE,HL		.
C670  CD4FC6		CALL	AC64F		.O.
C673  EB		EX	DE,HL		.
C674  228AC4		LD	(DC48A),HL	"..
C677  EB		EX	DE,HL		.
C678  E1		POP	HL		.
C679  1A		LD	A,(DE)		.
C67A  B7		OR	A		.
C67B  CA89C6		JP	Z,AC689		...
C67E  DE40		SBC	A,040H		.@
C680  47		LD	B,A		G
C681  13		INC	DE		.
C682  1A		LD	A,(DE)		.
C683  FE3A		CP	03AH		.:
C685  CA90C6		JP	Z,AC690		...
C688  1B		DEC	DE		.
C689  3AEFCB	AC689:	LD	A,(DCBEF)	:..
C68C  77		LD	(HL),A		w
C68D  C396C6		JP	AC696		...
		;
C690  78	AC690:	LD	A,B		x
C691  32F0CB		LD	(DCBF0),A	2..
C694  70		LD	(HL),B		p
C695  13		INC	DE		.
C696  0608	AC696:	LD	B,008H		..
C698  CD30C6	AC698:	CALL	AC630		.0.
C69B  CAB9C6		JP	Z,AC6B9		...
C69E  23		INC	HL		#
C69F  FE2A		CP	02AH		.*
C6A1  C2A9C6		JP	NZ,AC6A9	...
C6A4  363F		LD	(HL),03FH	6?
C6A6  C3ABC6		JP	AC6AB		...
		;
C6A9  77	AC6A9:	LD	(HL),A		w
C6AA  13		INC	DE		.
C6AB  05	AC6AB:	DEC	B		.
C6AC  C298C6		JP	NZ,AC698	...
C6AF  CD30C6	AC6AF:	CALL	AC630		.0.
C6B2  CAC0C6		JP	Z,AC6C0		...
C6B5  13		INC	DE		.
C6B6  C3AFC6		JP	AC6AF		...
		;
C6B9  23	AC6B9:	INC	HL		#
C6BA  3620		LD	(HL),020H	6 
C6BC  05		DEC	B		.
C6BD  C2B9C6		JP	NZ,AC6B9	...
C6C0  0603	AC6C0:	LD	B,003H		..
C6C2  FE2E		CP	02EH		..
C6C4  C2E9C6		JP	NZ,AC6E9	...
C6C7  13		INC	DE		.
C6C8  CD30C6	AC6C8:	CALL	AC630		.0.
C6CB  CAE9C6		JP	Z,AC6E9		...
C6CE  23		INC	HL		#
C6CF  FE2A		CP	02AH		.*
C6D1  C2D9C6		JP	NZ,AC6D9	...
C6D4  363F		LD	(HL),03FH	6?
C6D6  C3DBC6		JP	AC6DB		...
		;
C6D9  77	AC6D9:	LD	(HL),A		w
C6DA  13		INC	DE		.
C6DB  05	AC6DB:	DEC	B		.
C6DC  C2C8C6		JP	NZ,AC6C8	...
C6DF  CD30C6	AC6DF:	CALL	AC630		.0.
C6E2  CAF0C6		JP	Z,AC6F0		...
C6E5  13		INC	DE		.
C6E6  C3DFC6		JP	AC6DF		...
		;
C6E9  23	AC6E9:	INC	HL		#
C6EA  3620		LD	(HL),020H	6 
C6EC  05		DEC	B		.
C6ED  C2E9C6		JP	NZ,AC6E9	...
C6F0  0603	AC6F0:	LD	B,003H		..
C6F2  23	AC6F2:	INC	HL		#
C6F3  3600		LD	(HL),000H	6.
C6F5  05		DEC	B		.
C6F6  C2F2C6		JP	NZ,AC6F2	...
C6F9  EB		EX	DE,HL		.
C6FA  2288C4		LD	(DC488),HL	"..
C6FD  E1		POP	HL		.
C6FE  010B00		LD	BC,0000BH	...
C701  23	AC701:	INC	HL		#
C702  7E		LD	A,(HL)		~
C703  FE3F		CP	03FH		.?
C705  C209C7		JP	NZ,AC709	...
C708  04		INC	B		.
C709  0D	AC709:	DEC	C		.
C70A  C201C7		JP	NZ,AC701	...
C70D  78		LD	A,B		x
C70E  B7		OR	A		.
C70F  C9		RET			.
		;
		; >> NO EXECUTION PATH TO HERE <<
C710  DIR ERA TYPESAVEREN USER

C728  C8	TC728:	RET	Z		.
C729  1600		LD	D,000H		..
C72B  00		NOP			.
C72C  08		EX	AF,AF'		.
C72D  EB		EX	DE,HL		.
C72E  2110C7	AC72E:	LD	HL,TC710	!..
C731  0E00		LD	C,000H		..
C733  79	AC733:	LD	A,C		y
C734  FE06		CP	006H		..
C736  D0		RET	NC		.
C737  11CECB		LD	DE,DCBCE	...
C73A  0604		LD	B,004H		..
C73C  1A	AC73C:	LD	A,(DE)		.
C73D  BE		CP	(HL)		.
C73E  C24FC7		JP	NZ,AC74F	.O.
C741  13		INC	DE		.
C742  23		INC	HL		#
C743  05		DEC	B		.
C744  C23CC7		JP	NZ,AC73C	.<.
C747  1A		LD	A,(DE)		.
C748  FE20		CP	020H		. 
C74A  C254C7		JP	NZ,AC754	.T.
C74D  79		LD	A,C		y
C74E  C9		RET			.
		;
C74F  23	AC74F:	INC	HL		#
C750  05		DEC	B		.
C751  C24FC7		JP	NZ,AC74F	.O.
C754  0C	AC754:	INC	C		.
C755  C333C7		JP	AC733		.3.
		;
C758  AF	AC758:	XOR	A		.
C759  3207C4		LD	(AC407),A	2..
C75C  31ABCB	AC75C:	LD	SP,DCBAB	1..
C75F  C5		PUSH	BC		.
C760  79		LD	A,C		y
C761  1F		RRA			.
C762  1F		RRA			.
C763  1F		RRA			.
C764  1F		RRA			.
C765  E60F		AND	00FH		..
C767  5F		LD	E,A		_
C768  CD15C5		CALL	AC515		...
C76B  CDB8C4		CALL	AC4B8		...
C76E  32ABCB		LD	(DCBAB),A	2..
C771  C1		POP	BC		.
C772  79		LD	A,C		y
C773  E60F		AND	00FH		..
C775  32EFCB		LD	(DCBEF),A	2..
C778  CDBDC4		CALL	AC4BD		...
C77B  3A07C4		LD	A,(AC407)	:..
C77E  B7		OR	A		.
C77F  C298C7		JP	NZ,AC798	...
C782  31ABCB	AC782:	LD	SP,DCBAB	1..
C785  CD98C4		CALL	AC498		...
C788  CDD0C5		CALL	AC5D0		...
C78B  C641		ADD	A,041H		.A
C78D  CD8CC4		CALL	AC48C		...
C790  3E3E		LD	A,03EH		>>
C792  CD8CC4		CALL	AC48C		...
C795  CD39C5	AC795:	CALL	AC539		.9.
C798  118000	AC798:	LD	DE,00080H	...
C79B  CDD8C5		CALL	AC5D8		...
C79E  CDD0C5		CALL	AC5D0		...
C7A1  32EFCB		LD	(DCBEF),A	2..
C7A4  CD5EC6		CALL	AC65E		.^.
C7A7  C409C6		CALL	NZ,AC609	...
C7AA  3AF0CB		LD	A,(DCBF0)	:..
C7AD  B7		OR	A		.
C7AE  C2A5CA		JP	NZ,ACAA5	...
C7B1  CD2EC7		CALL	AC72E		...
C7B4  21C1C7		LD	HL,TC7C1	!..
C7B7  5F		LD	E,A		_
C7B8  1600		LD	D,000H		..
C7BA  19		ADD	HL,DE		.
C7BB  19		ADD	HL,DE		.
C7BC  7E		LD	A,(HL)		~
C7BD  23		INC	HL		#
C7BE  66		LD	H,(HL)		f
C7BF  6F		LD	L,A		o
C7C0  E9		JP	(HL)		.
		;
		; >> NO EXECUTION PATH TO HERE <<
C7C1  77	TC7C1:	LD	(HL),A		w
C7C2  C8		RET	Z		.
C7C3  1F		RRA			.
C7C4  C9		RET			.
		;
		; >> NO EXECUTION PATH TO HERE <<
C7C5  5D		LD	E,L		]
C7C6  C9		RET			.
		;
		; >> NO EXECUTION PATH TO HERE <<
C7C7  AD		XOR	L		.
C7C8  C9		RET			.
		;
		; >> NO EXECUTION PATH TO HERE <<
C7C9  10CA		DJNZ	AC795		..
C7CB  8E		ADC	A,(HL)		.
C7CC  CAA5CA		JP	Z,ACAA5		...
C7CF  21F376	AC7CF:	LD	HL,076F3H	!.v
C7D2  2200C4		LD	(DC400),HL	"..
C7D5  2100C4		LD	HL,DC400	!..
C7D8  E9		JP	(HL)		.
		;
C7D9  01DFC7	AC7D9:	LD	BC,TC7DF	...
C7DC  C3A7C4		JP	AC4A7		...
		;
		; >> NO EXECUTION PATH TO HERE <<
C7DF  52	TC7DF:	LD	D,D		R
C7E0  45		LD	B,L		E
C7E1  41		LD	B,C		A
C7E2  44		LD	B,H		D
C7E3  2045		JR	NZ,AC82A	 E
C7E5  52		LD	D,D		R
C7E6  52		LD	D,D		R
C7E7  4F		LD	C,A		O
C7E8  52		LD	D,D		R
C7E9  00		NOP			.
C7EA  01F0C7	AC7EA:	LD	BC,TC7F0	...
C7ED  C3A7C4		JP	AC4A7		...
		;
		; >> NO EXECUTION PATH TO HERE <<
C7F0  4E	TC7F0:	LD	C,(HL)		N
C7F1  4F		LD	C,A		O
C7F2  2046		JR	NZ,AC83A	 F
C7F4  49		LD	C,C		I
C7F5  4C		LD	C,H		L
C7F6  45		LD	B,L		E
C7F7  00		NOP			.
C7F8  CD5EC6	AC7F8:	CALL	AC65E		.^.
C7FB  3AF0CB		LD	A,(DCBF0)	:..
C7FE  B7		OR	A		.
C7FF  C209C6		JP	NZ,AC609	...
C802  21CECB		LD	HL,DCBCE	!..
C805  010B00		LD	BC,0000BH	...
C808  7E	AC808:	LD	A,(HL)		~
C809  FE20		CP	020H		. 
C80B  CA33C8		JP	Z,AC833		.3.
C80E  23		INC	HL		#
C80F  D630		SUB	030H		.0
C811  FE0A		CP	00AH		..
C813  D209C6		JP	NC,AC609	...
C816  57		LD	D,A		W
C817  78		LD	A,B		x
C818  E6E0		AND	0E0H		..
C81A  C209C6		JP	NZ,AC609	...
C81D  78		LD	A,B		x
C81E  07		RLCA			.
C81F  07		RLCA			.
C820  07		RLCA			.
C821  80		ADD	A,B		.
C822  DA09C6		JP	C,AC609		...
C825  80		ADD	A,B		.
C826  DA09C6		JP	C,AC609		...
C829  82		ADD	A,D		.
C82A  DA09C6	AC82A:	JP	C,AC609		...
C82D  47		LD	B,A		G
C82E  0D		DEC	C		.
C82F  C208C8		JP	NZ,AC808	...
C832  C9		RET			.
		;
C833  7E	AC833:	LD	A,(HL)		~
C834  FE20		CP	020H		. 
C836  C209C6		JP	NZ,AC609	...
C839  23		INC	HL		#
C83A  0D	AC83A:	DEC	C		.
C83B  C233C8		JP	NZ,AC833	.3.
C83E  78		LD	A,B		x
C83F  C9		RET			.
		;
C840  0603	AC840:	LD	B,003H		..
C842  7E	AC842:	LD	A,(HL)		~
C843  12		LD	(DE),A		.
C844  23		INC	HL		#
C845  13		INC	DE		.
C846  05		DEC	B		.
C847  C242C8		JP	NZ,AC842	.B.
C84A  C9		RET			.
		;
C84B  218000	AC84B:	LD	HL,00080H	!..
C84E  81		ADD	A,C		.
C84F  CD59C6		CALL	AC659		.Y.
C852  7E		LD	A,(HL)		~
C853  C9		RET			.
		;
C854  AF	AC854:	XOR	A		.
C855  32CDCB		LD	(DCBCD),A	2..
C858  3AF0CB		LD	A,(DCBF0)	:..
C85B  B7		OR	A		.
C85C  C8		RET	Z		.
C85D  3D		DEC	A		=
C85E  21EFCB		LD	HL,DCBEF	!..
C861  BE		CP	(HL)		.
C862  C8		RET	Z		.
C863  C3BDC4		JP	AC4BD		...
		;
C866  3AF0CB	AC866:	LD	A,(DCBF0)	:..
C869  B7		OR	A		.
C86A  C8		RET	Z		.
C86B  3D		DEC	A		=
C86C  21EFCB		LD	HL,DCBEF	!..
C86F  BE		CP	(HL)		.
C870  C8		RET	Z		.
C871  3AEFCB		LD	A,(DCBEF)	:..
C874  C3BDC4		JP	AC4BD		...
		;
		; >> NO EXECUTION PATH TO HERE <<
C877  CD5EC6		CALL	AC65E		.^.
C87A  CD54C8		CALL	AC854		.T.
C87D  21CECB		LD	HL,DCBCE	!..
C880  7E		LD	A,(HL)		~
C881  FE20		CP	020H		. 
C883  C28FC8		JP	NZ,AC88F	...
C886  060B		LD	B,00BH		..
C888  363F	AC888:	LD	(HL),03FH	6?
C88A  23		INC	HL		#
C88B  05		DEC	B		.
C88C  C288C8		JP	NZ,AC888	...
C88F  1E00	AC88F:	LD	E,000H		..
C891  D5		PUSH	DE		.
C892  CDE9C4		CALL	AC4E9		...
C895  CCEAC7		CALL	Z,AC7EA		...
C898  CA1BC9	AC898:	JP	Z,AC91B		...
C89B  3AEECB		LD	A,(DCBEE)	:..
C89E  0F		RRCA			.
C89F  0F		RRCA			.
C8A0  0F		RRCA			.
C8A1  E660		AND	060H		.`
C8A3  4F		LD	C,A		O
C8A4  3E0A		LD	A,00AH		>.
C8A6  CD4BC8		CALL	AC84B		.K.
C8A9  17		RLA			.
C8AA  DA0FC9		JP	C,AC90F		...
C8AD  D1		POP	DE		.
C8AE  7B		LD	A,E		{
C8AF  1C		INC	E		.
C8B0  D5		PUSH	DE		.
C8B1  E603		AND	003H		..
C8B3  F5		PUSH	AF		.
C8B4  C2CCC8		JP	NZ,AC8CC	...
C8B7  CD98C4		CALL	AC498		...
C8BA  C5		PUSH	BC		.
C8BB  CDD0C5		CALL	AC5D0		...
C8BE  C1		POP	BC		.
C8BF  C641		ADD	A,041H		.A
C8C1  CD92C4		CALL	AC492		...
C8C4  3E3A		LD	A,03AH		>:
C8C6  CD92C4		CALL	AC492		...
C8C9  C3D4C8		JP	AC8D4		...
		;
C8CC  CDA2C4	AC8CC:	CALL	AC4A2		...
C8CF  3E3A		LD	A,03AH		>:
C8D1  CD92C4		CALL	AC492		...
C8D4  CDA2C4	AC8D4:	CALL	AC4A2		...
C8D7  0601		LD	B,001H		..
C8D9  78	AC8D9:	LD	A,B		x
C8DA  CD4BC8		CALL	AC84B		.K.
C8DD  E67F		AND	07FH		..
C8DF  FE20		CP	020H		. 
C8E1  C2F9C8		JP	NZ,AC8F9	...
C8E4  F1		POP	AF		.
C8E5  F5		PUSH	AF		.
C8E6  FE03		CP	003H		..
C8E8  C2F7C8		JP	NZ,AC8F7	...
C8EB  3E09		LD	A,009H		>.
C8ED  CD4BC8		CALL	AC84B		.K.
C8F0  E67F		AND	07FH		..
C8F2  FE20		CP	020H		. 
C8F4  CA0EC9		JP	Z,AC90E		...
C8F7  3E20	AC8F7:	LD	A,020H		> 
C8F9  CD92C4	AC8F9:	CALL	AC492		...
C8FC  04		INC	B		.
C8FD  78		LD	A,B		x
C8FE  FE0C		CP	00CH		..
C900  D20EC9		JP	NC,AC90E	...
C903  FE09		CP	009H		..
C905  C2D9C8		JP	NZ,AC8D9	...
C908  CDA2C4		CALL	AC4A2		...
C90B  C3D9C8		JP	AC8D9		...
		;
C90E  F1	AC90E:	POP	AF		.
C90F  CDC2C5	AC90F:	CALL	AC5C2		...
C912  C21BC9		JP	NZ,AC91B	...
C915  CDE4C4		CALL	AC4E4		...
C918  C398C8		JP	AC898		...
		;
C91B  D1	AC91B:	POP	DE		.
C91C  C386CB		JP	ACB86		...
		;
		; >> NO EXECUTION PATH TO HERE <<
C91F  CD5EC6		CALL	AC65E		.^.
C922  FE0B		CP	00BH		..
C924  C242C9		JP	NZ,AC942	.B.
C927  0152C9		LD	BC,TC952	.R.
C92A  CDA7C4		CALL	AC4A7		...
C92D  CD39C5		CALL	AC539		.9.
C930  2107C4		LD	HL,AC407	!..
C933  35		DEC	(HL)		5
C934  C282C7		JP	NZ,AC782	...
C937  23		INC	HL		#
C938  7E		LD	A,(HL)		~
C939  FE59		CP	059H		.Y
C93B  C282C7		JP	NZ,AC782	...
C93E  23		INC	HL		#
C93F  2288C4		LD	(DC488),HL	"..
C942  CD54C8	AC942:	CALL	AC854		.T.
C945  11CDCB		LD	DE,DCBCD	...
C948  CDEFC4		CALL	AC4EF		...
C94B  3C		INC	A		<
C94C  CCEAC7		CALL	Z,AC7EA		...
C94F  C386CB		JP	ACB86		...
		;
		; >> NO EXECUTION PATH TO HERE <<
C952  ALL (Y/N)?
C95C  00		NOP			.
C95D  CD5EC6		CALL	AC65E		.^.
C960  C209C6		JP	NZ,AC609	...
C963  CD54C8		CALL	AC854		.T.
C966  CDD0C4		CALL	AC4D0		...
C969  CAA7C9		JP	Z,AC9A7		...
C96C  CD98C4		CALL	AC498		...
C96F  21F1CB		LD	HL,TCBF1	!..
C972  36FF		LD	(HL),0FFH	6.
C974  21F1CB	AC974:	LD	HL,TCBF1	!..
C977  7E		LD	A,(HL)		~
C978  FE80		CP	080H		..
C97A  DA87C9		JP	C,AC987		...
C97D  E5		PUSH	HL		.
C97E  CDFEC4		CALL	AC4FE		...
C981  E1		POP	HL		.
C982  C2A0C9		JP	NZ,AC9A0	...
C985  AF		XOR	A		.
C986  77		LD	(HL),A		w
C987  34	AC987:	INC	(HL)		4
C988  218000		LD	HL,00080H	!..
C98B  CD59C6		CALL	AC659		.Y.
C98E  7E		LD	A,(HL)		~
C98F  FE1A		CP	01AH		..
C991  CA86CB		JP	Z,ACB86		...
C994  CD8CC4		CALL	AC48C		...
C997  CDC2C5		CALL	AC5C2		...
C99A  C286CB		JP	NZ,ACB86	...
C99D  C374C9		JP	AC974		.t.
		;
C9A0  3D	AC9A0:	DEC	A		=
C9A1  CA86CB		JP	Z,ACB86		...
C9A4  CDD9C7		CALL	AC7D9		...
C9A7  CD66C8	AC9A7:	CALL	AC866		.f.
C9AA  C309C6		JP	AC609		...
		;
		; >> NO EXECUTION PATH TO HERE <<
C9AD  CDF8C7		CALL	AC7F8		...
C9B0  F5		PUSH	AF		.
C9B1  CD5EC6		CALL	AC65E		.^.
C9B4  C209C6		JP	NZ,AC609	...
C9B7  CD54C8		CALL	AC854		.T.
C9BA  11CDCB		LD	DE,DCBCD	...
C9BD  D5		PUSH	DE		.
C9BE  CDEFC4		CALL	AC4EF		...
C9C1  D1		POP	DE		.
C9C2  CD09C5		CALL	AC509		...
C9C5  CAFBC9		JP	Z,AC9FB		...
C9C8  AF		XOR	A		.
C9C9  32EDCB		LD	(DCBED),A	2..
C9CC  F1		POP	AF		.
C9CD  6F		LD	L,A		o
C9CE  2600		LD	H,000H		&.
C9D0  29		ADD	HL,HL		)
C9D1  110001		LD	DE,00100H	...
C9D4  7C	AC9D4:	LD	A,H		|
C9D5  B5		OR	L		.
C9D6  CAF1C9		JP	Z,AC9F1		...
C9D9  2B		DEC	HL		+
C9DA  E5		PUSH	HL		.
C9DB  218000		LD	HL,00080H	!..
C9DE  19		ADD	HL,DE		.
C9DF  E5		PUSH	HL		.
C9E0  CDD8C5		CALL	AC5D8		...
C9E3  11CDCB		LD	DE,DCBCD	...
C9E6  CD04C5		CALL	AC504		...
C9E9  D1		POP	DE		.
C9EA  E1		POP	HL		.
C9EB  C2FBC9		JP	NZ,AC9FB	...
C9EE  C3D4C9		JP	AC9D4		...
		;
C9F1  11CDCB	AC9F1:	LD	DE,DCBCD	...
C9F4  CDDAC4		CALL	AC4DA		...
C9F7  3C		INC	A		<
C9F8  C201CA		JP	NZ,ACA01	...
C9FB  0107CA	AC9FB:	LD	BC,TCA07	...
C9FE  CDA7C4		CALL	AC4A7		...
CA01  CDD5C5	ACA01:	CALL	AC5D5		...
CA04  C386CB		JP	ACB86		...
		;
		; >> NO EXECUTION PATH TO HERE <<
CA07  NO SPACE
CA0F  00		NOP			.
CA10  CD5EC6		CALL	AC65E		.^.
CA13  C209C6		JP	NZ,AC609	...
CA16  3AF0CB		LD	A,(DCBF0)	:..
CA19  F5		PUSH	AF		.
CA1A  CD54C8		CALL	AC854		.T.
CA1D  CDE9C4		CALL	AC4E9		...
CA20  C279CA		JP	NZ,ACA79	.y.
CA23  21CDCB		LD	HL,DCBCD	!..
CA26  11DDCB		LD	DE,DCBDD	...
CA29  0610		LD	B,010H		..
CA2B  CD42C8		CALL	AC842		.B.
CA2E  2A88C4		LD	HL,(DC488)	*..
CA31  EB		EX	DE,HL		.
CA32  CD4FC6		CALL	AC64F		.O.
CA35  FE3D		CP	03DH		.=
CA37  CA3FCA		JP	Z,ACA3F		.?.
CA3A  FE5F		CP	05FH		._
CA3C  C273CA		JP	NZ,ACA73	.s.
CA3F  EB	ACA3F:	EX	DE,HL		.
CA40  23		INC	HL		#
CA41  2288C4		LD	(DC488),HL	"..
CA44  CD5EC6		CALL	AC65E		.^.
CA47  C273CA		JP	NZ,ACA73	.s.
CA4A  F1		POP	AF		.
CA4B  47		LD	B,A		G
CA4C  21F0CB		LD	HL,DCBF0	!..
CA4F  7E		LD	A,(HL)		~
CA50  B7		OR	A		.
CA51  CA59CA		JP	Z,ACA59		.Y.
CA54  B8		CP	B		.
CA55  70		LD	(HL),B		p
CA56  C273CA		JP	NZ,ACA73	.s.
CA59  70	ACA59:	LD	(HL),B		p
CA5A  AF		XOR	A		.
CA5B  32CDCB		LD	(DCBCD),A	2..
CA5E  CDE9C4	ACA5E:	CALL	AC4E9		...
CA61  CA6DCA		JP	Z,ACA6D		.m.
CA64  11CDCB		LD	DE,DCBCD	...
CA67  CD0EC5		CALL	AC50E		...
CA6A  C386CB		JP	ACB86		...
		;
CA6D  CDEAC7	ACA6D:	CALL	AC7EA		...
CA70  C386CB		JP	ACB86		...
		;
CA73  CD66C8	ACA73:	CALL	AC866		.f.
CA76  C309C6		JP	AC609		...
		;
CA79  0182CA	ACA79:	LD	BC,TCA82	...
CA7C  CDA7C4		CALL	AC4A7		...
CA7F  C386CB		JP	ACB86		...
		;
		; >> NO EXECUTION PATH TO HERE <<
CA82  FILE EXISTS
CA8D  00		NOP			.
CA8E  CDF8C7		CALL	AC7F8		...
CA91  FE10		CP	010H		..
CA93  D209C6		JP	NC,AC609	...
CA96  5F		LD	E,A		_
CA97  3ACECB		LD	A,(DCBCE)	:..
CA9A  FE20		CP	020H		. 
CA9C  CA09C6		JP	Z,AC609		...
CA9F  CD15C5		CALL	AC515		...
CAA2  C389CB		JP	ACB89		...
		;
CAA5  CDF5C5	ACAA5:	CALL	AC5F5		...
CAA8  3ACECB		LD	A,(DCBCE)	:..
CAAB  FE20		CP	020H		. 
CAAD  C2C4CA		JP	NZ,ACAC4	...
CAB0  3AF0CB		LD	A,(DCBF0)	:..
CAB3  B7		OR	A		.
CAB4  CA89CB		JP	Z,ACB89		...
CAB7  3D		DEC	A		=
CAB8  32EFCB		LD	(DCBEF),A	2..
CABB  CD29C5		CALL	AC529		.).
CABE  CDBDC4		CALL	AC4BD		...
CAC1  C389CB		JP	ACB89		...
		;
CAC4  11D6CB	ACAC4:	LD	DE,TCBD6	...
CAC7  1A		LD	A,(DE)		.
CAC8  FE20		CP	020H		. 
CACA  C209C6		JP	NZ,AC609	...
CACD  D5	ACACD:	PUSH	DE		.
CACE  CD54C8		CALL	AC854		.T.
CAD1  D1		POP	DE		.
CAD2  2183CB		LD	HL,TCB83	!..
CAD5  CD40C8		CALL	AC840		.@.
CAD8  CDD0C4		CALL	AC4D0		...
CADB  CA6BCB		JP	Z,ACB6B		.k.
CADE  210001		LD	HL,00100H	!..
CAE1  E5	ACAE1:	PUSH	HL		.
CAE2  EB		EX	DE,HL		.
CAE3  CDD8C5		CALL	AC5D8		...
CAE6  11CDCB		LD	DE,DCBCD	...
CAE9  CDF9C4		CALL	AC4F9		...
CAEC  C201CB		JP	NZ,ACB01	...
CAEF  E1		POP	HL		.
CAF0  118000		LD	DE,00080H	...
CAF3  19		ADD	HL,DE		.
CAF4  1100C4		LD	DE,DC400	...
CAF7  7D		LD	A,L		}
CAF8  93		SUB	E		.
CAF9  7C		LD	A,H		|
CAFA  9A		SBC	A,D		.
CAFB  D271CB		JP	NC,ACB71	.q.
CAFE  C3E1CA		JP	ACAE1		...
		;
CB01  E1	ACB01:	POP	HL		.
CB02  3D		DEC	A		=
CB03  C271CB		JP	NZ,ACB71	.q.
CB06  CD66C8		CALL	AC866		.f.
CB09  CD5EC6		CALL	AC65E		.^.
CB0C  21F0CB		LD	HL,DCBF0	!..
CB0F  E5		PUSH	HL		.
CB10  7E		LD	A,(HL)		~
CB11  32CDCB		LD	(DCBCD),A	2..
CB14  3E10		LD	A,010H		>.
CB16  CD60C6		CALL	AC660		.`.
CB19  E1		POP	HL		.
CB1A  7E		LD	A,(HL)		~
CB1B  32DDCB		LD	(DCBDD),A	2..
CB1E  AF		XOR	A		.
CB1F  32EDCB		LD	(DCBED),A	2..
CB22  115C00		LD	DE,0005CH	.\.
CB25  21CDCB		LD	HL,DCBCD	!..
CB28  0621		LD	B,021H		.!
CB2A  CD42C8		CALL	AC842		.B.
CB2D  2108C4		LD	HL,TC408	!..
CB30  7E	ACB30:	LD	A,(HL)		~
CB31  B7		OR	A		.
CB32  CA3ECB		JP	Z,ACB3E		.>.
CB35  FE20		CP	020H		. 
CB37  CA3ECB		JP	Z,ACB3E		.>.
CB3A  23		INC	HL		#
CB3B  C330CB		JP	ACB30		.0.
		;
CB3E  0600	ACB3E:	LD	B,000H		..
CB40  118100		LD	DE,00081H	...
CB43  7E	ACB43:	LD	A,(HL)		~
CB44  12		LD	(DE),A		.
CB45  B7		OR	A		.
CB46  CA4FCB		JP	Z,ACB4F		.O.
CB49  04		INC	B		.
CB4A  23		INC	HL		#
CB4B  13		INC	DE		.
CB4C  C343CB		JP	ACB43		.C.
		;
CB4F  78	ACB4F:	LD	A,B		x
CB50  328000		LD	(Y0080),A	2..
CB53  CD98C4		CALL	AC498		...
CB56  CDD5C5		CALL	AC5D5		...
CB59  CD1AC5		CALL	AC51A		...
CB5C  CD0001		CALL	X0100		...
CB5F  31ABCB		LD	SP,DCBAB	1..
CB62  CD29C5		CALL	AC529		.).
CB65  CDBDC4		CALL	AC4BD		...
CB68  C382C7		JP	AC782		...
		;
CB6B  CD66C8	ACB6B:	CALL	AC866		.f.
CB6E  C309C6		JP	AC609		...
		;
CB71  017ACB	ACB71:	LD	BC,TCB7A	.z.
CB74  CDA7C4		CALL	AC4A7		...
CB77  C386CB		JP	ACB86		...
		;
		; >> NO EXECUTION PATH TO HERE <<
CB7A  BAD LOAD.COM

CB86  CD66C8	ACB86:	CALL	AC866		.f.
CB89  CD5EC6	ACB89:	CALL	AC65E		.^.
CB8C  3ACECB		LD	A,(DCBCE)	:..
CB8F  D620		SUB	020H		. 
CB91  21F0CB		LD	HL,DCBF0	!..
CB94  B6		OR	(HL)		.
CB95  C209C6		JP	NZ,AC609	...
CB98  C382C7		JP	AC782		...
		;
		; >> NO EXECUTION PATH TO HERE <<
CB9B  00		NOP			.
...
CBA2  00		NOP			.
CBA3  96		SUB	(HL)		.
CBA4  C41DC5		CALL	NZ,AC51D	...
CBA7  A4		AND	H		.
CBA8  C5		PUSH	BC		.
CBA9  98		SBC	A,B		.
CBAA  C7		RST	000H		.
CBAB  00	DCBAB:	NOP			.
CBAC  00	TCBAC:	NOP			.
CBAD  $$$     SUB

CBB8  00		NOP			.
...
CBEE  00	DCBEE:	NOP			.
CBEF  02	DCBEF:		(Default Disk is saved here)
CBF0  00	DCBF0:	NOP			.
...
CBFF  00		NOP			.
CC00  C8	TCC00:	RET	Z		.
CC01  1600		LD	D,000H		..
CC03  00		NOP			.
CC04  08		EX	AF,AF'		.
CC05  EB		EX	DE,HL		.
CC06  C311CC		JP	ACC11		...
		;
CC09  99	ACC09:	SBC	A,C		.
CC0A  CCA5CC		CALL	Z,ACCA5		...
CC0D  AB	TCC0D:	XOR	E		.
CC0E  CCB1CC		CALL	Z,ACCB1		...
CC11  EB	ACC11:	EX	DE,HL		.
CC12  2243CF		LD	(DCF43),HL	"C.
CC15  EB		EX	DE,HL		.
CC16  7B		LD	A,E		{
CC17  32D6D9		LD	(DD9D6),A	2..
CC1A  210000		LD	HL,00000H	!..
CC1D  2245CF		LD	(DCF45),HL	"E.
CC20  39		ADD	HL,SP		9
CC21  220FCF		LD	(DCF0F),HL	"..
CC24  3141CF		LD	SP,DCF41	1A.
CC27  AF		XOR	A		.
CC28  32E0D9		LD	(DD9E0),A	2..
CC2B  32DED9		LD	(DD9DE),A	2..
CC2E  2174D9		LD	HL,AD974	!t.
CC31  E5		PUSH	HL		.
CC32  79		LD	A,C		y
CC33  FE29		CP	029H		.)
CC35  D0		RET	NC		.
CC36  4B		LD	C,E		K
CC37  2147CC		LD	HL,TCC47	!G.
CC3A  5F		LD	E,A		_
CC3B  1600		LD	D,000H		..
CC3D  19		ADD	HL,DE		.
CC3E  19		ADD	HL,DE		.
CC3F  5E		LD	E,(HL)		^
CC40  23		INC	HL		#
CC41  56		LD	D,(HL)		V
CC42  2A43CF		LD	HL,(DCF43)	*C.
CC45  EB		EX	DE,HL		.
CC46  E9		JP	(HL)		.
		;
		; >> NO EXECUTION PATH TO HERE <<
CC47  03	TCC47:	INC	BC		.
CC48  DAC8CE		JP	C,ACEC8		...
CC4B  90		SUB	B		.
CC4C  CDCECE		CALL	ACECE		...
CC4F  12		LD	(DE),A		.
CC50  DA0FDA		JP	C,XDA0F		...
CC53  D4CEED		CALL	NC,XEDCE	...
CC56  CEF3		ADC	A,0F3H		..
CC58  CEF8		ADC	A,0F8H		..
CC5A  CEE1		ADC	A,0E1H		..
CC5C  CDFECE		CALL	ACEFE		...
CC5F  7E		LD	A,(HL)		~
CC60  D8		RET	C		.
CC61  83		ADD	A,E		.
CC62  D8		RET	C		.
CC63  45		LD	B,L		E
CC64  D8		RET	C		.
CC65  9C		SBC	A,H		.
CC66  D8		RET	C		.
CC67  A5		AND	L		.
CC68  D8		RET	C		.
CC69  AB		XOR	E		.
CC6A  D8		RET	C		.
CC6B  C8		RET	Z		.
CC6C  D8		RET	C		.
CC6D  D7		RST	010H		.
CC6E  D8		RET	C		.
CC6F  E0		RET	PO		.
CC70  D8		RET	C		.
CC71  E6D8		AND	0D8H		..
CC73  ECD8F5		CALL	PE,XF5D8	...
CC76  D8		RET	C		.
CC77  FED8		CP	0D8H		..
CC79  04		INC	B		.
CC7A  D9		EXX			.
CC7B  0A		LD	A,(BC)		.
CC7C  D9		EXX			.
CC7D  11D92C		LD	DE,02CD9H	..,
CC80  D1		POP	DE		.
CC81  17		RLA			.
CC82  D9		EXX			.
CC83  1D		DEC	E		.
CC84  D9		EXX			.
CC85  26D9		LD	H,0D9H		&.
CC87  2D		DEC	L		-
CC88  D9		EXX			.
CC89  41		LD	B,C		A
CC8A  D9		EXX			.
CC8B  47		LD	B,A		G
CC8C  D9		EXX			.
CC8D  4D		LD	C,L		M
CC8E  D9		EXX			.
CC8F  0ED8		LD	C,0D8H		..
CC91  53		LD	D,E		S
CC92  D9		EXX			.
CC93  04		INC	B		.
CC94  CF		RST	008H		.
CC95  04		INC	B		.
CC96  CF		RST	008H		.
CC97  9B		SBC	A,E		.
CC98  D9		EXX			.
CC99  21CACC		LD	HL,TCCCA	!..
CC9C  CDE5CC		CALL	ACCE5		...
CC9F  FE03		CP	003H		..
CCA1  CA0000		JP	Z,X0000		...
CCA4  C9		RET			.
		;
CCA5  21D5CC	ACCA5:	LD	HL,TCCD5	!..
CCA8  C3B4CC		JP	ACCB4		...
		;
		; >> NO EXECUTION PATH TO HERE <<
CCAB  21E1CC		LD	HL,TCCE1	!..
CCAE  C3B4CC		JP	ACCB4		...
		;
CCB1  21DCCC	ACCB1:	LD	HL,TCCDC	!..
CCB4  CDE5CC	ACCB4:	CALL	ACCE5		...
CCB7  C30000		JP	X0000		...
		;
		; >> NO EXECUTION PATH TO HERE <<
CCBA  Bdos Err On  : $

CCCA  Bad Sector$

CCD5  Select$

CCDC  File R/O$

CCE5  E5	ACCE5:	PUSH	HL		.
CCE6  CDC9CD		CALL	ACDC9		...
CCE9  3A42CF		LD	A,(DCF42)	:B.
CCEC  C641		ADD	A,041H		.A
CCEE  32C6CC		LD	(DCCC6),A	2..
CCF1  01BACC		LD	BC,TCCBA	...
CCF4  CDD3CD		CALL	ACDD3		...
CCF7  C1		POP	BC		.
CCF8  CDD3CD		CALL	ACDD3		...
CCFB  210ECF	ACCFB:	LD	HL,DCF0E	!..
CCFE  7E		LD	A,(HL)		~
CCFF  3600		LD	(HL),000H	6.
CD01  B7		OR	A		.
CD02  C0		RET	NZ		.
CD03  C309DA		JP	XDA09		...
		;
CD06  CDFBCC	ACD06:	CALL	ACCFB		...
CD09  CD14CD		CALL	ACD14		...
CD0C  D8		RET	C		.
CD0D  F5		PUSH	AF		.
CD0E  4F		LD	C,A		O
CD0F  CD90CD		CALL	ACD90		...
CD12  F1		POP	AF		.
CD13  C9	ACD13:	RET			.
		;
CD14  FE0D	ACD14:	CP	00DH		..
CD16  C8		RET	Z		.
CD17  FE0A		CP	00AH		..
CD19  C8		RET	Z		.
CD1A  FE09		CP	009H		..
CD1C  C8		RET	Z		.
CD1D  FE08		CP	008H		..
CD1F  C8		RET	Z		.
CD20  FE20		CP	020H		. 
CD22  C9	ACD22:	RET			.
		;
CD23  3A0ECF	ACD23:	LD	A,(DCF0E)	:..
CD26  B7		OR	A		.
CD27  C245CD		JP	NZ,ACD45	.E.
CD2A  CD06DA		CALL	XDA06		...
CD2D  E601		AND	001H		..
CD2F  C8		RET	Z		.
CD30  CD09DA		CALL	XDA09		...
CD33  FE13		CP	013H		..
CD35  C242CD		JP	NZ,ACD42	.B.
CD38  CD09DA		CALL	XDA09		...
CD3B  FE03		CP	003H		..
CD3D  CA0000		JP	Z,X0000		...
CD40  AF		XOR	A		.
CD41  C9		RET			.
		;
CD42  320ECF	ACD42:	LD	(DCF0E),A	2..
CD45  3E01	ACD45:	LD	A,001H		>.
CD47  C9		RET			.
		;
CD48  3A0ACF	ACD48:	LD	A,(DCF0A)	:..
CD4B  B7		OR	A		.
CD4C  C262CD		JP	NZ,ACD62	.b.
CD4F  C5		PUSH	BC		.
CD50  CD23CD		CALL	ACD23		.#.
CD53  C1		POP	BC		.
CD54  C5		PUSH	BC		.
CD55  CD0CDA		CALL	XDA0C		...
CD58  C1		POP	BC		.
CD59  C5		PUSH	BC		.
CD5A  3A0DCF		LD	A,(DCF0D)	:..
CD5D  B7		OR	A		.
CD5E  C40FDA		CALL	NZ,XDA0F	...
CD61  C1		POP	BC		.
CD62  79	ACD62:	LD	A,C		y
CD63  210CCF		LD	HL,DCF0C	!..
CD66  FE7F		CP	07FH		..
CD68  C8		RET	Z		.
CD69  34		INC	(HL)		4
CD6A  FE20		CP	020H		. 
CD6C  D0		RET	NC		.
CD6D  35		DEC	(HL)		5
CD6E  7E		LD	A,(HL)		~
CD6F  B7		OR	A		.
CD70  C8		RET	Z		.
CD71  79		LD	A,C		y
CD72  FE08		CP	008H		..
CD74  C279CD		JP	NZ,ACD79	.y.
CD77  35		DEC	(HL)		5
CD78  C9		RET			.
		;
CD79  FE0A	ACD79:	CP	00AH		..
CD7B  C0		RET	NZ		.
CD7C  3600		LD	(HL),000H	6.
CD7E  C9		RET			.
		;
CD7F  79	ACD7F:	LD	A,C		y
CD80  CD14CD		CALL	ACD14		...
CD83  D290CD		JP	NC,ACD90	...
CD86  F5		PUSH	AF		.
CD87  0E5E		LD	C,05EH		.^
CD89  CD48CD		CALL	ACD48		.H.
CD8C  F1		POP	AF		.
CD8D  F640		OR	040H		.@
CD8F  4F		LD	C,A		O
CD90  79	ACD90:	LD	A,C		y
CD91  FE09		CP	009H		..
CD93  C248CD		JP	NZ,ACD48	.H.
CD96  0E20	ACD96:	LD	C,020H		. 
CD98  CD48CD		CALL	ACD48		.H.
CD9B  3A0CCF		LD	A,(DCF0C)	:..
CD9E  E607		AND	007H		..
CDA0  C296CD		JP	NZ,ACD96	...
CDA3  C9		RET			.
		;
CDA4  CDACCD	ACDA4:	CALL	ACDAC		...
CDA7  0E20		LD	C,020H		. 
CDA9  CD0CDA		CALL	XDA0C		...
CDAC  0E08	ACDAC:	LD	C,008H		..
CDAE  C30CDA		JP	XDA0C		...
		;
CDB1  0E23	ACDB1:	LD	C,023H		.#
CDB3  CD48CD		CALL	ACD48		.H.
CDB6  CDC9CD		CALL	ACDC9		...
CDB9  3A0CCF	ACDB9:	LD	A,(DCF0C)	:..
CDBC  210BCF		LD	HL,DCF0B	!..
CDBF  BE		CP	(HL)		.
CDC0  D0		RET	NC		.
CDC1  0E20		LD	C,020H		. 
CDC3  CD48CD		CALL	ACD48		.H.
CDC6  C3B9CD		JP	ACDB9		...
		;
CDC9  0E0D	ACDC9:	LD	C,00DH		..
CDCB  CD48CD		CALL	ACD48		.H.
CDCE  0E0A		LD	C,00AH		..
CDD0  C348CD		JP	ACD48		.H.
		;
CDD3  0A	ACDD3:	LD	A,(BC)		.
CDD4  FE24		CP	024H		.$
CDD6  C8		RET	Z		.
CDD7  03		INC	BC		.
CDD8  C5		PUSH	BC		.
CDD9  4F		LD	C,A		O
CDDA  CD90CD		CALL	ACD90		...
CDDD  C1		POP	BC		.
CDDE  C3D3CD		JP	ACDD3		...
		;
CDE1  3A0CCF	ACDE1:	LD	A,(DCF0C)	:..
CDE4  320BCF		LD	(DCF0B),A	2..
CDE7  2A43CF		LD	HL,(DCF43)	*C.
CDEA  4E		LD	C,(HL)		N
CDEB  23		INC	HL		#
CDEC  E5		PUSH	HL		.
CDED  0600		LD	B,000H		..
CDEF  C5	ACDEF:	PUSH	BC		.
CDF0  E5		PUSH	HL		.
CDF1  CDFBCC	ACDF1:	CALL	ACCFB		...
CDF4  E67F		AND	07FH		..
CDF6  E1		POP	HL		.
CDF7  C1		POP	BC		.
CDF8  FE0D		CP	00DH		..
CDFA  CAC1CE		JP	Z,ACEC1		...
CDFD  FE0A		CP	00AH		..
CDFF  CAC1CE		JP	Z,ACEC1		...
CE02  FE08		CP	008H		..
CE04  C216CE		JP	NZ,ACE16	...
CE07  78		LD	A,B		x
CE08  B7		OR	A		.
CE09  CAEFCD		JP	Z,ACDEF		...
CE0C  05		DEC	B		.
CE0D  3A0CCF		LD	A,(DCF0C)	:..
CE10  320ACF		LD	(DCF0A),A	2..
CE13  C370CE		JP	ACE70		.p.
		;
CE16  FE7F	ACE16:	CP	07FH		..
CE18  C226CE		JP	NZ,ACE26	.&.
CE1B  78		LD	A,B		x
CE1C  B7		OR	A		.
CE1D  CAEFCD		JP	Z,ACDEF		...
CE20  7E		LD	A,(HL)		~
CE21  05		DEC	B		.
CE22  2B		DEC	HL		+
CE23  C3A9CE		JP	ACEA9		...
		;
CE26  FE05	ACE26:	CP	005H		..
CE28  C237CE		JP	NZ,ACE37	.7.
CE2B  C5		PUSH	BC		.
CE2C  E5		PUSH	HL		.
CE2D  CDC9CD		CALL	ACDC9		...
CE30  AF		XOR	A		.
CE31  320BCF		LD	(DCF0B),A	2..
CE34  C3F1CD		JP	ACDF1		...
		;
CE37  FE10	ACE37:	CP	010H		..
CE39  C248CE		JP	NZ,ACE48	.H.
CE3C  E5		PUSH	HL		.
CE3D  210DCF		LD	HL,DCF0D	!..
CE40  3E01		LD	A,001H		>.
CE42  96		SUB	(HL)		.
CE43  77		LD	(HL),A		w
CE44  E1		POP	HL		.
CE45  C3EFCD		JP	ACDEF		...
		;
CE48  FE18	ACE48:	CP	018H		..
CE4A  C25FCE		JP	NZ,ACE5F	._.
CE4D  E1		POP	HL		.
CE4E  3A0BCF	ACE4E:	LD	A,(DCF0B)	:..
CE51  210CCF		LD	HL,DCF0C	!..
CE54  BE		CP	(HL)		.
CE55  D2E1CD		JP	NC,ACDE1	...
CE58  35		DEC	(HL)		5
CE59  CDA4CD		CALL	ACDA4		...
CE5C  C34ECE		JP	ACE4E		.N.
		;
CE5F  FE15	ACE5F:	CP	015H		..
CE61  C26BCE		JP	NZ,ACE6B	.k.
CE64  CDB1CD		CALL	ACDB1		...
CE67  E1		POP	HL		.
CE68  C3E1CD		JP	ACDE1		...
		;
CE6B  FE12	ACE6B:	CP	012H		..
CE6D  C2A6CE		JP	NZ,ACEA6	...
CE70  C5	ACE70:	PUSH	BC		.
CE71  CDB1CD		CALL	ACDB1		...
CE74  C1		POP	BC		.
CE75  E1		POP	HL		.
CE76  E5		PUSH	HL		.
CE77  C5		PUSH	BC		.
CE78  78	ACE78:	LD	A,B		x
CE79  B7		OR	A		.
CE7A  CA8ACE		JP	Z,ACE8A		...
CE7D  23		INC	HL		#
CE7E  4E		LD	C,(HL)		N
CE7F  05		DEC	B		.
CE80  C5		PUSH	BC		.
CE81  E5		PUSH	HL		.
CE82  CD7FCD		CALL	ACD7F		...
CE85  E1		POP	HL		.
CE86  C1		POP	BC		.
CE87  C378CE		JP	ACE78		.x.
		;
CE8A  E5	ACE8A:	PUSH	HL		.
CE8B  3A0ACF		LD	A,(DCF0A)	:..
CE8E  B7		OR	A		.
CE8F  CAF1CD		JP	Z,ACDF1		...
CE92  210CCF		LD	HL,DCF0C	!..
CE95  96		SUB	(HL)		.
CE96  320ACF		LD	(DCF0A),A	2..
CE99  CDA4CD	ACE99:	CALL	ACDA4		...
CE9C  210ACF		LD	HL,DCF0A	!..
CE9F  35		DEC	(HL)		5
CEA0  C299CE		JP	NZ,ACE99	...
CEA3  C3F1CD		JP	ACDF1		...
		;
CEA6  23	ACEA6:	INC	HL		#
CEA7  77		LD	(HL),A		w
CEA8  04		INC	B		.
CEA9  C5	ACEA9:	PUSH	BC		.
CEAA  E5		PUSH	HL		.
CEAB  4F		LD	C,A		O
CEAC  CD7FCD		CALL	ACD7F		...
CEAF  E1		POP	HL		.
CEB0  C1		POP	BC		.
CEB1  7E		LD	A,(HL)		~
CEB2  FE03		CP	003H		..
CEB4  78		LD	A,B		x
CEB5  C2BDCE		JP	NZ,ACEBD	...
CEB8  FE01		CP	001H		..
CEBA  CA0000		JP	Z,X0000		...
CEBD  B9	ACEBD:	CP	C		.
CEBE  DAEFCD		JP	C,ACDEF		...
CEC1  E1	ACEC1:	POP	HL		.
CEC2  70		LD	(HL),B		p
CEC3  0E0D		LD	C,00DH		..
CEC5  C348CD		JP	ACD48		.H.
		;
CEC8  CD06CD	ACEC8:	CALL	ACD06		...
CECB  C301CF		JP	ACF01		...
		;
CECE  CD15DA	ACECE:	CALL	XDA15		...
CED1  C301CF		JP	ACF01		...
		;
		; >> NO EXECUTION PATH TO HERE <<
CED4  79		LD	A,C		y
CED5  3C		INC	A		<
CED6  CAE0CE		JP	Z,ACEE0		...
CED9  3C		INC	A		<
CEDA  CA06DA		JP	Z,XDA06		...
CEDD  C30CDA		JP	XDA0C		...
		;
CEE0  CD06DA	ACEE0:	CALL	XDA06		...
CEE3  B7		OR	A		.
CEE4  CA91D9		JP	Z,AD991		...
CEE7  CD09DA		CALL	XDA09		...
CEEA  C301CF		JP	ACF01		...
		;
		; >> NO EXECUTION PATH TO HERE <<
CEED  3A0300		LD	A,(Y0003)	:..
CEF0  C301CF		JP	ACF01		...
		;
		; >> NO EXECUTION PATH TO HERE <<
CEF3  210300		LD	HL,00003H	!..
CEF6  71		LD	(HL),C		q
CEF7  C9		RET			.
		;
		; >> NO EXECUTION PATH TO HERE <<
CEF8  EB		EX	DE,HL		.
CEF9  4D		LD	C,L		M
CEFA  44		LD	B,H		D
CEFB  C3D3CD		JP	ACDD3		...
		;
CEFE  CD23CD	ACEFE:	CALL	ACD23		.#.
CF01  3245CF	ACF01:	LD	(DCF45),A	2E.
CF04  C9		RET			.
		;
CF05  3E01	ACF05:	LD	A,001H		>.
CF07  C301CF		JP	ACF01		...
		;
		; >> NO EXECUTION PATH TO HERE <<
CF0A  00	DCF0A:	NOP			.
CF0B  02	DCF0B:	LD	(BC),A		.
CF0C  02	DCF0C:	LD	(BC),A		.
CF0D  00	DCF0D:	NOP			.
CF0E  00	DCF0E:	NOP			.
CF0F  A7	DCF0F:	AND	A		.
CF10  CB00		RLC	B		..
CF12  00		NOP			.
...
CF2E  00		NOP			.
CF2F  F8		RET	M		.
CF30  DB1D		IN	A,(01DH)	..
CF32  D0		RET	NC		.
CF33  10DC		DJNZ	ACF11		..
CF35  C0		RET	NZ		.
CF36  DBF4		IN	A,(0F4H)	..
CF38  CD07C4		CALL	AC407		...
CF3B  4D		LD	C,L		M
CF3C  00		NOP			.
CF3D  07		RLCA			.
CF3E  C474D9		CALL	NZ,AD974	.t.
CF41  00	DCF41:	NOP			.
CF42  02	DCF42:	LD	(BC),A		.
CF43  06C4	DCF43:	LD	B,0C4H		..
CF45  00	DCF45:	NOP			.
CF46  00		NOP			.
CF47  210BCC	ACF47:	LD	HL,TCC0B	!..
CF4A  5E	ACF4A:	LD	E,(HL)		^
CF4B  23		INC	HL		#
CF4C  56		LD	D,(HL)		V
CF4D  EB		EX	DE,HL		.
CF4E  E9		JP	(HL)		.
		;
CF4F  0C	ACF4F:	INC	C		.
CF50  0D	ACF50:	DEC	C		.
CF51  C8		RET	Z		.
CF52  1A		LD	A,(DE)		.
CF53  77		LD	(HL),A		w
CF54  13		INC	DE		.
CF55  23		INC	HL		#
CF56  C350CF		JP	ACF50		.P.
		;
CF59  3A42CF	ACF59:	LD	A,(DCF42)	:B.
CF5C  4F		LD	C,A		O
CF5D  CD1BDA		CALL	XDA1B		...
CF60  7C		LD	A,H		|
CF61  B5		OR	L		.
CF62  C8		RET	Z		.
CF63  5E		LD	E,(HL)		^
CF64  23		INC	HL		#
CF65  56		LD	D,(HL)		V
CF66  23		INC	HL		#
CF67  22B3D9		LD	(DD9B3),HL	"..
CF6A  23		INC	HL		#
CF6B  23		INC	HL		#
CF6C  22B5D9		LD	(DD9B5),HL	"..
CF6F  23		INC	HL		#
CF70  23		INC	HL		#
CF71  22B7D9		LD	(DD9B7),HL	"..
CF74  23		INC	HL		#
CF75  23		INC	HL		#
CF76  EB		EX	DE,HL		.
CF77  22D0D9		LD	(DD9D0),HL	"..
CF7A  21B9D9		LD	HL,DD9B9	!..
CF7D  0E08		LD	C,008H		..
CF7F  CD4FCF		CALL	ACF4F		.O.
CF82  2ABBD9		LD	HL,(DD9BB)	*..
CF85  EB		EX	DE,HL		.
CF86  21C1D9		LD	HL,DD9C1	!..
CF89  0E0F		LD	C,00FH		..
CF8B  CD4FCF		CALL	ACF4F		.O.
CF8E  2AC6D9		LD	HL,(DD9C6)	*..
CF91  7C		LD	A,H		|
CF92  21DDD9		LD	HL,DD9DD	!..
CF95  36FF		LD	(HL),0FFH	6.
CF97  B7		OR	A		.
CF98  CA9DCF		JP	Z,ACF9D		...
CF9B  3600		LD	(HL),000H	6.
CF9D  3EFF	ACF9D:	LD	A,0FFH		>.
CF9F  B7		OR	A		.
CFA0  C9		RET			.
		;
CFA1  CD18DA	ACFA1:	CALL	XDA18		...
CFA4  AF		XOR	A		.
CFA5  2AB5D9		LD	HL,(DD9B5)	*..
CFA8  77		LD	(HL),A		w
CFA9  23		INC	HL		#
CFAA  77		LD	(HL),A		w
CFAB  2AB7D9		LD	HL,(DD9B7)	*..
CFAE  77		LD	(HL),A		w
CFAF  23		INC	HL		#
CFB0  77		LD	(HL),A		w
CFB1  C9		RET			.
		;
CFB2  CD27DA	ACFB2:	CALL	XDA27		.'.
CFB5  C3BBCF		JP	ACFBB		...
		;
CFB8  CD2ADA	ACFB8:	CALL	XDA2A		.*.
CFBB  B7	ACFBB:	OR	A		.
CFBC  C8		RET	Z		.
CFBD  2109CC		LD	HL,ACC09	!..
CFC0  C34ACF		JP	ACF4A		.J.
		;
CFC3  2AEAD9	ACFC3:	LD	HL,(DD9EA)	*..
CFC6  0E02		LD	C,002H		..
CFC8  CDEAD0		CALL	AD0EA		...
CFCB  22E5D9		LD	(DD9E5),HL	"..
CFCE  22ECD9		LD	(DD9EC),HL	"..
CFD1  21E5D9	ACFD1:	LD	HL,DD9E5	!..
CFD4  4E		LD	C,(HL)		N
CFD5  23		INC	HL		#
CFD6  46		LD	B,(HL)		F
CFD7  2AB7D9		LD	HL,(DD9B7)	*..
CFDA  5E		LD	E,(HL)		^
CFDB  23		INC	HL		#
CFDC  56		LD	D,(HL)		V
CFDD  2AB5D9		LD	HL,(DD9B5)	*..
CFE0  7E		LD	A,(HL)		~
CFE1  23		INC	HL		#
CFE2  66		LD	H,(HL)		f
CFE3  6F		LD	L,A		o
CFE4  79	ACFE4:	LD	A,C		y
CFE5  93		SUB	E		.
CFE6  78		LD	A,B		x
CFE7  9A		SBC	A,D		.
CFE8  D2FACF		JP	NC,ACFFA	...
CFEB  E5		PUSH	HL		.
CFEC  2AC1D9		LD	HL,(DD9C1)	*..
CFEF  7B		LD	A,E		{
CFF0  95		SUB	L		.
CFF1  5F		LD	E,A		_
CFF2  7A		LD	A,D		z
CFF3  9C		SBC	A,H		.
CFF4  57		LD	D,A		W
CFF5  E1		POP	HL		.
CFF6  2B		DEC	HL		+
CFF7  C3E4CF		JP	ACFE4		...
		;
CFFA  E5	ACFFA:	PUSH	HL		.
CFFB  2AC1D9		LD	HL,(DD9C1)	*..
CFFE  19		ADD	HL,DE		.
CFFF  DA0FD0		JP	C,AD00F		...
D002  79		LD	A,C		y
D003  95		SUB	L		.
D004  78		LD	A,B		x
D005  9C		SBC	A,H		.
D006  DA0FD0		JP	C,AD00F		...
D009  EB		EX	DE,HL		.
D00A  E1		POP	HL		.
D00B  23		INC	HL		#
D00C  C3FACF		JP	ACFFA		...
		;
D00F  E1	AD00F:	POP	HL		.
D010  C5		PUSH	BC		.
D011  D5		PUSH	DE		.
D012  E5		PUSH	HL		.
D013  EB		EX	DE,HL		.
D014  2ACED9		LD	HL,(DD9CE)	*..
D017  19		ADD	HL,DE		.
D018  44		LD	B,H		D
D019  4D		LD	C,L		M
D01A  CD1EDA		CALL	XDA1E		...
D01D  D1		POP	DE		.
D01E  2AB5D9		LD	HL,(DD9B5)	*..
D021  73		LD	(HL),E		s
D022  23		INC	HL		#
D023  72		LD	(HL),D		r
D024  D1		POP	DE		.
D025  2AB7D9		LD	HL,(DD9B7)	*..
D028  73		LD	(HL),E		s
D029  23		INC	HL		#
D02A  72		LD	(HL),D		r
D02B  C1		POP	BC		.
D02C  79		LD	A,C		y
D02D  93		SUB	E		.
D02E  4F		LD	C,A		O
D02F  78		LD	A,B		x
D030  9A		SBC	A,D		.
D031  47		LD	B,A		G
D032  2AD0D9		LD	HL,(DD9D0)	*..
D035  EB		EX	DE,HL		.
D036  CD30DA		CALL	XDA30		.0.
D039  4D		LD	C,L		M
D03A  44		LD	B,H		D
D03B  C321DA		JP	XDA21		.!.
		;
D03E  21C3D9	AD03E:	LD	HL,DD9C3	!..
D041  4E		LD	C,(HL)		N
D042  3AE3D9		LD	A,(DD9E3)	:..
D045  B7	AD045:	OR	A		.
D046  1F		RRA			.
D047  0D		DEC	C		.
D048  C245D0		JP	NZ,AD045	.E.
D04B  47		LD	B,A		G
D04C  3E08		LD	A,008H		>.
D04E  96		SUB	(HL)		.
D04F  4F		LD	C,A		O
D050  3AE2D9		LD	A,(DD9E2)	:..
D053  0D	AD053:	DEC	C		.
D054  CA5CD0		JP	Z,AD05C		.\.
D057  B7		OR	A		.
D058  17		RLA			.
D059  C353D0		JP	AD053		.S.
		;
D05C  80	AD05C:	ADD	A,B		.
D05D  C9		RET			.
		;
D05E  2A43CF	AD05E:	LD	HL,(DCF43)	*C.
D061  111000		LD	DE,00010H	...
D064  19		ADD	HL,DE		.
D065  09		ADD	HL,BC		.
D066  3ADDD9		LD	A,(DD9DD)	:..
D069  B7		OR	A		.
D06A  CA71D0		JP	Z,AD071		.q.
D06D  6E		LD	L,(HL)		n
D06E  2600		LD	H,000H		&.
D070  C9		RET			.
		;
D071  09	AD071:	ADD	HL,BC		.
D072  5E		LD	E,(HL)		^
D073  23		INC	HL		#
D074  56		LD	D,(HL)		V
D075  EB		EX	DE,HL		.
D076  C9		RET			.
		;
D077  CD3ED0	AD077:	CALL	AD03E		.>.
D07A  4F		LD	C,A		O
D07B  0600		LD	B,000H		..
D07D  CD5ED0		CALL	AD05E		.^.
D080  22E5D9		LD	(DD9E5),HL	"..
D083  C9		RET			.
		;
D084  2AE5D9	AD084:	LD	HL,(DD9E5)	*..
D087  7D		LD	A,L		}
D088  B4		OR	H		.
D089  C9		RET			.
		;
D08A  3AC3D9	AD08A:	LD	A,(DD9C3)	:..
D08D  2AE5D9		LD	HL,(DD9E5)	*..
D090  29	AD090:	ADD	HL,HL		)
D091  3D		DEC	A		=
D092  C290D0		JP	NZ,AD090	...
D095  22E7D9		LD	(DD9E7),HL	"..
D098  3AC4D9		LD	A,(DD9C4)	:..
D09B  4F		LD	C,A		O
D09C  3AE3D9		LD	A,(DD9E3)	:..
D09F  A1		AND	C		.
D0A0  B5		OR	L		.
D0A1  6F		LD	L,A		o
D0A2  22E5D9		LD	(DD9E5),HL	"..
D0A5  C9		RET			.
		;
D0A6  2A43CF	AD0A6:	LD	HL,(DCF43)	*C.
D0A9  110C00		LD	DE,0000CH	...
D0AC  19		ADD	HL,DE		.
D0AD  C9		RET			.
		;
D0AE  2A43CF	AD0AE:	LD	HL,(DCF43)	*C.
D0B1  110F00		LD	DE,0000FH	...
D0B4  19		ADD	HL,DE		.
D0B5  EB		EX	DE,HL		.
D0B6  211100		LD	HL,00011H	!..
D0B9  19		ADD	HL,DE		.
D0BA  C9		RET			.
		;
D0BB  CDAED0	AD0BB:	CALL	AD0AE		...
D0BE  7E		LD	A,(HL)		~
D0BF  32E3D9		LD	(DD9E3),A	2..
D0C2  EB		EX	DE,HL		.
D0C3  7E		LD	A,(HL)		~
D0C4  32E1D9		LD	(DD9E1),A	2..
D0C7  CDA6D0		CALL	AD0A6		...
D0CA  3AC5D9		LD	A,(DD9C5)	:..
D0CD  A6		AND	(HL)		.
D0CE  32E2D9		LD	(DD9E2),A	2..
D0D1  C9		RET			.
		;
D0D2  CDAED0	AD0D2:	CALL	AD0AE		...
D0D5  3AD5D9		LD	A,(DD9D5)	:..
D0D8  FE02		CP	002H		..
D0DA  C2DED0		JP	NZ,AD0DE	...
D0DD  AF		XOR	A		.
D0DE  4F	AD0DE:	LD	C,A		O
D0DF  3AE3D9		LD	A,(DD9E3)	:..
D0E2  81		ADD	A,C		.
D0E3  77		LD	(HL),A		w
D0E4  EB		EX	DE,HL		.
D0E5  3AE1D9		LD	A,(DD9E1)	:..
D0E8  77		LD	(HL),A		w
D0E9  C9		RET			.
		;
D0EA  0C	AD0EA:	INC	C		.
D0EB  0D	AD0EB:	DEC	C		.
D0EC  C8		RET	Z		.
D0ED  7C		LD	A,H		|
D0EE  B7		OR	A		.
D0EF  1F		RRA			.
D0F0  67		LD	H,A		g
D0F1  7D		LD	A,L		}
D0F2  1F		RRA			.
D0F3  6F		LD	L,A		o
D0F4  C3EBD0		JP	AD0EB		...
		;
D0F7  0E80	AD0F7:	LD	C,080H		..
D0F9  2AB9D9		LD	HL,(DD9B9)	*..
D0FC  AF		XOR	A		.
D0FD  86	AD0FD:	ADD	A,(HL)		.
D0FE  23		INC	HL		#
D0FF  0D		DEC	C		.
D100  C2FDD0		JP	NZ,AD0FD	...
D103  C9		RET			.
		;
D104  0C	AD104:	INC	C		.
D105  0D	AD105:	DEC	C		.
D106  C8		RET	Z		.
D107  29		ADD	HL,HL		)
D108  C305D1		JP	AD105		...
		;
D10B  C5	AD10B:	PUSH	BC		.
D10C  3A42CF		LD	A,(DCF42)	:B.
D10F  4F		LD	C,A		O
D110  210100		LD	HL,00001H	!..
D113  CD04D1		CALL	AD104		...
D116  C1		POP	BC		.
D117  79		LD	A,C		y
D118  B5		OR	L		.
D119  6F		LD	L,A		o
D11A  78		LD	A,B		x
D11B  B4		OR	H		.
D11C  67		LD	H,A		g
D11D  C9		RET			.
		;
D11E  2AADD9	AD11E:	LD	HL,(DD9AD)	*..
D121  3A42CF		LD	A,(DCF42)	:B.
D124  4F		LD	C,A		O
D125  CDEAD0		CALL	AD0EA		...
D128  7D		LD	A,L		}
D129  E601		AND	001H		..
D12B  C9		RET			.
		;
D12C  21ADD9	AD12C:	LD	HL,DD9AD	!..
D12F  4E		LD	C,(HL)		N
D130  23		INC	HL		#
D131  46		LD	B,(HL)		F
D132  CD0BD1		CALL	AD10B		...
D135  22ADD9		LD	(DD9AD),HL	"..
D138  2AC8D9		LD	HL,(DD9C8)	*..
D13B  23		INC	HL		#
D13C  EB		EX	DE,HL		.
D13D  2AB3D9		LD	HL,(DD9B3)	*..
D140  73		LD	(HL),E		s
D141  23		INC	HL		#
D142  72		LD	(HL),D		r
D143  C9		RET			.
		;
D144  CD5ED1	AD144:	CALL	AD15E		.^.
D147  110900	AD147:	LD	DE,00009H	...
D14A  19		ADD	HL,DE		.
D14B  7E		LD	A,(HL)		~
D14C  17		RLA			.
D14D  D0		RET	NC		.
D14E  210FCC		LD	HL,TCC0F	!..
D151  C34ACF		JP	ACF4A		.J.
		;
D154  CD1ED1	AD154:	CALL	AD11E		...
D157  C8		RET	Z		.
D158  210DCC		LD	HL,TCC0D	!..
D15B  C34ACF		JP	ACF4A		.J.
		;
D15E  2AB9D9	AD15E:	LD	HL,(DD9B9)	*..
D161  3AE9D9		LD	A,(DD9E9)	:..
D164  85	AD164:	ADD	A,L		.
D165  6F		LD	L,A		o
D166  D0		RET	NC		.
D167  24		INC	H		$
D168  C9		RET			.
		;
D169  2A43CF	AD169:	LD	HL,(DCF43)	*C.
D16C  110E00		LD	DE,0000EH	...
D16F  19		ADD	HL,DE		.
D170  7E		LD	A,(HL)		~
D171  C9		RET			.
		;
D172  CD69D1	AD172:	CALL	AD169		.i.
D175  3600		LD	(HL),000H	6.
D177  C9		RET			.
		;
D178  CD69D1	AD178:	CALL	AD169		.i.
D17B  F680		OR	080H		..
D17D  77		LD	(HL),A		w
D17E  C9		RET			.
		;
D17F  2AEAD9	AD17F:	LD	HL,(DD9EA)	*..
D182  EB		EX	DE,HL		.
D183  2AB3D9		LD	HL,(DD9B3)	*..
D186  7B		LD	A,E		{
D187  96		SUB	(HL)		.
D188  23		INC	HL		#
D189  7A		LD	A,D		z
D18A  9E		SBC	A,(HL)		.
D18B  C9		RET			.
		;
D18C  CD7FD1	AD18C:	CALL	AD17F		...
D18F  D8		RET	C		.
D190  13		INC	DE		.
D191  72		LD	(HL),D		r
D192  2B		DEC	HL		+
D193  73		LD	(HL),E		s
D194  C9		RET			.
		;
D195  7B	AD195:	LD	A,E		{
D196  95		SUB	L		.
D197  6F		LD	L,A		o
D198  7A		LD	A,D		z
D199  9C		SBC	A,H		.
D19A  67		LD	H,A		g
D19B  C9		RET			.
		;
D19C  0EFF	AD19C:	LD	C,0FFH		..
D19E  2AECD9	AD19E:	LD	HL,(DD9EC)	*..
D1A1  EB		EX	DE,HL		.
D1A2  2ACCD9		LD	HL,(DD9CC)	*..
D1A5  CD95D1		CALL	AD195		...
D1A8  D0		RET	NC		.
D1A9  C5		PUSH	BC		.
D1AA  CDF7D0		CALL	AD0F7		...
D1AD  2ABDD9		LD	HL,(DD9BD)	*..
D1B0  EB		EX	DE,HL		.
D1B1  2AECD9		LD	HL,(DD9EC)	*..
D1B4  19		ADD	HL,DE		.
D1B5  C1		POP	BC		.
D1B6  0C		INC	C		.
D1B7  CAC4D1		JP	Z,AD1C4		...
D1BA  BE		CP	(HL)		.
D1BB  C8		RET	Z		.
D1BC  CD7FD1		CALL	AD17F		...
D1BF  D0		RET	NC		.
D1C0  CD2CD1		CALL	AD12C		.,.
D1C3  C9		RET			.
		;
D1C4  77	AD1C4:	LD	(HL),A		w
D1C5  C9		RET			.
		;
D1C6  CD9CD1	AD1C6:	CALL	AD19C		...
D1C9  CDE0D1		CALL	AD1E0		...
D1CC  0E01		LD	C,001H		..
D1CE  CDB8CF		CALL	ACFB8		...
D1D1  C3DAD1		JP	AD1DA		...
		;
D1D4  CDE0D1	AD1D4:	CALL	AD1E0		...
D1D7  CDB2CF		CALL	ACFB2		...
D1DA  21B1D9	AD1DA:	LD	HL,DD9B1	!..
D1DD  C3E3D1		JP	AD1E3		...
		;
D1E0  21B9D9	AD1E0:	LD	HL,DD9B9	!..
D1E3  4E	AD1E3:	LD	C,(HL)		N
D1E4  23		INC	HL		#
D1E5  46		LD	B,(HL)		F
D1E6  C324DA		JP	XDA24		.$.
		;
D1E9  2AB9D9	AD1E9:	LD	HL,(DD9B9)	*..
D1EC  EB		EX	DE,HL		.
D1ED  2AB1D9		LD	HL,(DD9B1)	*..
D1F0  0E80		LD	C,080H		..
D1F2  C34FCF		JP	ACF4F		.O.
		;
D1F5  21EAD9	AD1F5:	LD	HL,DD9EA	!..
D1F8  7E		LD	A,(HL)		~
D1F9  23		INC	HL		#
D1FA  BE		CP	(HL)		.
D1FB  C0		RET	NZ		.
D1FC  3C		INC	A		<
D1FD  C9		RET			.
		;
D1FE  21FFFF	AD1FE:	LD	HL,0FFFFH	!..
D201  22EAD9		LD	(DD9EA),HL	"..
D204  C9		RET			.
		;
D205  2AC8D9	AD205:	LD	HL,(DD9C8)	*..
D208  EB		EX	DE,HL		.
D209  2AEAD9		LD	HL,(DD9EA)	*..
D20C  23		INC	HL		#
D20D  22EAD9		LD	(DD9EA),HL	"..
D210  CD95D1		CALL	AD195		...
D213  D219D2		JP	NC,AD219	...
D216  C3FED1		JP	AD1FE		...
		;
D219  3AEAD9	AD219:	LD	A,(DD9EA)	:..
D21C  E603		AND	003H		..
D21E  0605		LD	B,005H		..
D220  87	AD220:	ADD	A,A		.
D221  05		DEC	B		.
D222  C220D2		JP	NZ,AD220	. .
D225  32E9D9		LD	(DD9E9),A	2..
D228  B7		OR	A		.
D229  C0		RET	NZ		.
D22A  C5		PUSH	BC		.
D22B  CDC3CF		CALL	ACFC3		...
D22E  CDD4D1		CALL	AD1D4		...
D231  C1		POP	BC		.
D232  C39ED1		JP	AD19E		...
		;
D235  79	AD235:	LD	A,C		y
D236  E607		AND	007H		..
D238  3C		INC	A		<
D239  5F		LD	E,A		_
D23A  57		LD	D,A		W
D23B  79		LD	A,C		y
D23C  0F		RRCA			.
D23D  0F		RRCA			.
D23E  0F		RRCA			.
D23F  E61F		AND	01FH		..
D241  4F		LD	C,A		O
D242  78		LD	A,B		x
D243  87		ADD	A,A		.
D244  87		ADD	A,A		.
D245  87		ADD	A,A		.
D246  87		ADD	A,A		.
D247  87		ADD	A,A		.
D248  B1		OR	C		.
D249  4F		LD	C,A		O
D24A  78		LD	A,B		x
D24B  0F		RRCA			.
D24C  0F		RRCA			.
D24D  0F		RRCA			.
D24E  E61F		AND	01FH		..
D250  47		LD	B,A		G
D251  2ABFD9		LD	HL,(DD9BF)	*..
D254  09		ADD	HL,BC		.
D255  7E		LD	A,(HL)		~
D256  07	AD256:	RLCA			.
D257  1D		DEC	E		.
D258  C256D2		JP	NZ,AD256	.V.
D25B  C9		RET			.
		;
D25C  D5	AD25C:	PUSH	DE		.
D25D  CD35D2		CALL	AD235		.5.
D260  E6FE		AND	0FEH		..
D262  C1		POP	BC		.
D263  B1		OR	C		.
D264  0F	AD264:	RRCA			.
D265  15		DEC	D		.
D266  C264D2		JP	NZ,AD264	.d.
D269  77		LD	(HL),A		w
D26A  C9		RET			.
		;
D26B  CD5ED1	AD26B:	CALL	AD15E		.^.
D26E  111000		LD	DE,00010H	...
D271  19		ADD	HL,DE		.
D272  C5		PUSH	BC		.
D273  0E11		LD	C,011H		..
D275  D1	AD275:	POP	DE		.
D276  0D		DEC	C		.
D277  C8		RET	Z		.
D278  D5		PUSH	DE		.
D279  3ADDD9		LD	A,(DD9DD)	:..
D27C  B7		OR	A		.
D27D  CA88D2		JP	Z,AD288		...
D280  C5		PUSH	BC		.
D281  E5		PUSH	HL		.
D282  4E		LD	C,(HL)		N
D283  0600		LD	B,000H		..
D285  C38ED2		JP	AD28E		...
		;
D288  0D	AD288:	DEC	C		.
D289  C5		PUSH	BC		.
D28A  4E		LD	C,(HL)		N
D28B  23		INC	HL		#
D28C  46		LD	B,(HL)		F
D28D  E5		PUSH	HL		.
D28E  79	AD28E:	LD	A,C		y
D28F  B0		OR	B		.
D290  CA9DD2		JP	Z,AD29D		...
D293  2AC6D9		LD	HL,(DD9C6)	*..
D296  7D		LD	A,L		}
D297  91		SUB	C		.
D298  7C		LD	A,H		|
D299  98		SBC	A,B		.
D29A  D45CD2		CALL	NC,AD25C	.\.
D29D  E1	AD29D:	POP	HL		.
D29E  23		INC	HL		#
D29F  C1		POP	BC		.
D2A0  C375D2		JP	AD275		.u.
		;
D2A3  2AC6D9	AD2A3:	LD	HL,(DD9C6)	*..
D2A6  0E03		LD	C,003H		..
D2A8  CDEAD0		CALL	AD0EA		...
D2AB  23		INC	HL		#
D2AC  44		LD	B,H		D
D2AD  4D		LD	C,L		M
D2AE  2ABFD9		LD	HL,(DD9BF)	*..
D2B1  3600	AD2B1:	LD	(HL),000H	6.
D2B3  23		INC	HL		#
D2B4  0B		DEC	BC		.
D2B5  78		LD	A,B		x
D2B6  B1		OR	C		.
D2B7  C2B1D2		JP	NZ,AD2B1	...
D2BA  2ACAD9		LD	HL,(DD9CA)	*..
D2BD  EB		EX	DE,HL		.
D2BE  2ABFD9		LD	HL,(DD9BF)	*..
D2C1  73		LD	(HL),E		s
D2C2  23		INC	HL		#
D2C3  72		LD	(HL),D		r
D2C4  CDA1CF		CALL	ACFA1		...
D2C7  2AB3D9		LD	HL,(DD9B3)	*..
D2CA  3603		LD	(HL),003H	6.
D2CC  23		INC	HL		#
D2CD  3600		LD	(HL),000H	6.
D2CF  CDFED1		CALL	AD1FE		...
D2D2  0EFF	AD2D2:	LD	C,0FFH		..
D2D4  CD05D2		CALL	AD205		...
D2D7  CDF5D1		CALL	AD1F5		...
D2DA  C8		RET	Z		.
D2DB  CD5ED1		CALL	AD15E		.^.
D2DE  3EE5		LD	A,0E5H		>.
D2E0  BE		CP	(HL)		.
D2E1  CAD2D2		JP	Z,AD2D2		...
D2E4  3A41CF		LD	A,(DCF41)	:A.
D2E7  BE		CP	(HL)		.
D2E8  C2F6D2		JP	NZ,AD2F6	...
D2EB  23		INC	HL		#
D2EC  7E		LD	A,(HL)		~
D2ED  D624		SUB	024H		.$
D2EF  C2F6D2		JP	NZ,AD2F6	...
D2F2  3D		DEC	A		=
D2F3  3245CF		LD	(DCF45),A	2E.
D2F6  0E01	AD2F6:	LD	C,001H		..
D2F8  CD6BD2		CALL	AD26B		.k.
D2FB  CD8CD1		CALL	AD18C		...
D2FE  C3D2D2		JP	AD2D2		...
		;
D301  3AD4D9	AD301:	LD	A,(DD9D4)	:..
D304  C301CF		JP	ACF01		...
		;
D307  C5	AD307:	PUSH	BC		.
D308  F5		PUSH	AF		.
D309  3AC5D9		LD	A,(DD9C5)	:..
D30C  2F		CPL			/
D30D  47		LD	B,A		G
D30E  79		LD	A,C		y
D30F  A0		AND	B		.
D310  4F		LD	C,A		O
D311  F1		POP	AF		.
D312  A0		AND	B		.
D313  91		SUB	C		.
D314  E61F		AND	01FH		..
D316  C1		POP	BC		.
D317  C9		RET			.
		;
D318  3EFF	AD318:	LD	A,0FFH		>.
D31A  32D4D9		LD	(DD9D4),A	2..
D31D  21D8D9		LD	HL,DD9D8	!..
D320  71		LD	(HL),C		q
D321  2A43CF		LD	HL,(DCF43)	*C.
D324  22D9D9		LD	(DD9D9),HL	"..
D327  CDFED1		CALL	AD1FE		...
D32A  CDA1CF		CALL	ACFA1		...
D32D  0E00	AD32D:	LD	C,000H		..
D32F  CD05D2		CALL	AD205		...
D332  CDF5D1		CALL	AD1F5		...
D335  CA94D3		JP	Z,AD394		...
D338  2AD9D9		LD	HL,(DD9D9)	*..
D33B  EB		EX	DE,HL		.
D33C  1A		LD	A,(DE)		.
D33D  FEE5		CP	0E5H		..
D33F  CA4AD3		JP	Z,AD34A		.J.
D342  D5		PUSH	DE		.
D343  CD7FD1		CALL	AD17F		...
D346  D1		POP	DE		.
D347  D294D3		JP	NC,AD394	...
D34A  CD5ED1	AD34A:	CALL	AD15E		.^.
D34D  3AD8D9		LD	A,(DD9D8)	:..
D350  4F		LD	C,A		O
D351  0600		LD	B,000H		..
D353  79	AD353:	LD	A,C		y
D354  B7		OR	A		.
D355  CA83D3		JP	Z,AD383		...
D358  1A		LD	A,(DE)		.
D359  FE3F		CP	03FH		.?
D35B  CA7CD3		JP	Z,AD37C		.|.
D35E  78		LD	A,B		x
D35F  FE0D		CP	00DH		..
D361  CA7CD3		JP	Z,AD37C		.|.
D364  FE0C		CP	00CH		..
D366  1A		LD	A,(DE)		.
D367  CA73D3		JP	Z,AD373		.s.
D36A  96		SUB	(HL)		.
D36B  E67F		AND	07FH		..
D36D  C22DD3		JP	NZ,AD32D	.-.
D370  C37CD3		JP	AD37C		.|.
		;
D373  C5	AD373:	PUSH	BC		.
D374  4E		LD	C,(HL)		N
D375  CD07D3		CALL	AD307		...
D378  C1		POP	BC		.
D379  C22DD3		JP	NZ,AD32D	.-.
D37C  13	AD37C:	INC	DE		.
D37D  23		INC	HL		#
D37E  04		INC	B		.
D37F  0D		DEC	C		.
D380  C353D3		JP	AD353		.S.
		;
D383  3AEAD9	AD383:	LD	A,(DD9EA)	:..
D386  E603		AND	003H		..
D388  3245CF		LD	(DCF45),A	2E.
D38B  21D4D9		LD	HL,DD9D4	!..
D38E  7E		LD	A,(HL)		~
D38F  17		RLA			.
D390  D0		RET	NC		.
D391  AF		XOR	A		.
D392  77		LD	(HL),A		w
D393  C9		RET			.
		;
D394  CDFED1	AD394:	CALL	AD1FE		...
D397  3EFF		LD	A,0FFH		>.
D399  C301CF		JP	ACF01		...
		;
D39C  CD54D1	AD39C:	CALL	AD154		.T.
D39F  0E0C		LD	C,00CH		..
D3A1  CD18D3		CALL	AD318		...
D3A4  CDF5D1	AD3A4:	CALL	AD1F5		...
D3A7  C8		RET	Z		.
D3A8  CD44D1		CALL	AD144		.D.
D3AB  CD5ED1		CALL	AD15E		.^.
D3AE  36E5		LD	(HL),0E5H	6.
D3B0  0E00		LD	C,000H		..
D3B2  CD6BD2		CALL	AD26B		.k.
D3B5  CDC6D1		CALL	AD1C6		...
D3B8  CD2DD3		CALL	AD32D		.-.
D3BB  C3A4D3		JP	AD3A4		...
		;
D3BE  50	AD3BE:	LD	D,B		P
D3BF  59		LD	E,C		Y
D3C0  79	AD3C0:	LD	A,C		y
D3C1  B0		OR	B		.
D3C2  CAD1D3		JP	Z,AD3D1		...
D3C5  0B		DEC	BC		.
D3C6  D5		PUSH	DE		.
D3C7  C5		PUSH	BC		.
D3C8  CD35D2		CALL	AD235		.5.
D3CB  1F		RRA			.
D3CC  D2ECD3		JP	NC,AD3EC	...
D3CF  C1		POP	BC		.
D3D0  D1		POP	DE		.
D3D1  2AC6D9	AD3D1:	LD	HL,(DD9C6)	*..
D3D4  7B		LD	A,E		{
D3D5  95		SUB	L		.
D3D6  7A		LD	A,D		z
D3D7  9C		SBC	A,H		.
D3D8  D2F4D3		JP	NC,AD3F4	...
D3DB  13		INC	DE		.
D3DC  C5		PUSH	BC		.
D3DD  D5		PUSH	DE		.
D3DE  42		LD	B,D		B
D3DF  4B		LD	C,E		K
D3E0  CD35D2		CALL	AD235		.5.
D3E3  1F		RRA			.
D3E4  D2ECD3		JP	NC,AD3EC	...
D3E7  D1		POP	DE		.
D3E8  C1		POP	BC		.
D3E9  C3C0D3		JP	AD3C0		...
		;
D3EC  17	AD3EC:	RLA			.
D3ED  3C		INC	A		<
D3EE  CD64D2		CALL	AD264		.d.
D3F1  E1		POP	HL		.
D3F2  D1		POP	DE		.
D3F3  C9		RET			.
		;
D3F4  79	AD3F4:	LD	A,C		y
D3F5  B0		OR	B		.
D3F6  C2C0D3		JP	NZ,AD3C0	...
D3F9  210000		LD	HL,00000H	!..
D3FC  C9		RET			.
		;
D3FD  0E00	AD3FD:	LD	C,000H		..
D3FF  1E20		LD	E,020H		. 
D401  D5	AD401:	PUSH	DE		.
D402  0600		LD	B,000H		..
D404  2A43CF		LD	HL,(DCF43)	*C.
D407  09		ADD	HL,BC		.
D408  EB		EX	DE,HL		.
D409  CD5ED1		CALL	AD15E		.^.
D40C  C1		POP	BC		.
D40D  CD4FCF		CALL	ACF4F		.O.
D410  CDC3CF	AD410:	CALL	ACFC3		...
D413  C3C6D1		JP	AD1C6		...
		;
D416  CD54D1	AD416:	CALL	AD154		.T.
D419  0E0C		LD	C,00CH		..
D41B  CD18D3		CALL	AD318		...
D41E  2A43CF		LD	HL,(DCF43)	*C.
D421  7E		LD	A,(HL)		~
D422  111000		LD	DE,00010H	...
D425  19		ADD	HL,DE		.
D426  77		LD	(HL),A		w
D427  CDF5D1	AD427:	CALL	AD1F5		...
D42A  C8		RET	Z		.
D42B  CD44D1		CALL	AD144		.D.
D42E  0E10		LD	C,010H		..
D430  1E0C		LD	E,00CH		..
D432  CD01D4		CALL	AD401		...
D435  CD2DD3		CALL	AD32D		.-.
D438  C327D4		JP	AD427		.'.
		;
D43B  0E0C	AD43B:	LD	C,00CH		..
D43D  CD18D3		CALL	AD318		...
D440  CDF5D1	AD440:	CALL	AD1F5		...
D443  C8		RET	Z		.
D444  0E00		LD	C,000H		..
D446  1E0C		LD	E,00CH		..
D448  CD01D4		CALL	AD401		...
D44B  CD2DD3		CALL	AD32D		.-.
D44E  C340D4		JP	AD440		.@.
		;
D451  0E0F	AD451:	LD	C,00FH		..
D453  CD18D3		CALL	AD318		...
D456  CDF5D1		CALL	AD1F5		...
D459  C8		RET	Z		.
D45A  CDA6D0	AD45A:	CALL	AD0A6		...
D45D  7E		LD	A,(HL)		~
D45E  F5		PUSH	AF		.
D45F  E5		PUSH	HL		.
D460  CD5ED1		CALL	AD15E		.^.
D463  EB		EX	DE,HL		.
D464  2A43CF		LD	HL,(DCF43)	*C.
D467  0E20		LD	C,020H		. 
D469  D5		PUSH	DE		.
D46A  CD4FCF		CALL	ACF4F		.O.
D46D  CD78D1		CALL	AD178		.x.
D470  D1		POP	DE		.
D471  210C00		LD	HL,0000CH	!..
D474  19		ADD	HL,DE		.
D475  4E		LD	C,(HL)		N
D476  210F00		LD	HL,0000FH	!..
D479  19		ADD	HL,DE		.
D47A  46		LD	B,(HL)		F
D47B  E1		POP	HL		.
D47C  F1		POP	AF		.
D47D  77		LD	(HL),A		w
D47E  79		LD	A,C		y
D47F  BE		CP	(HL)		.
D480  78		LD	A,B		x
D481  CA8BD4		JP	Z,AD48B		...
D484  3E00		LD	A,000H		>.
D486  DA8BD4		JP	C,AD48B		...
D489  3E80		LD	A,080H		>.
D48B  2A43CF	AD48B:	LD	HL,(DCF43)	*C.
D48E  110F00		LD	DE,0000FH	...
D491  19		ADD	HL,DE		.
D492  77		LD	(HL),A		w
D493  C9		RET			.
		;
D494  7E	AD494:	LD	A,(HL)		~
D495  23		INC	HL		#
D496  B6		OR	(HL)		.
D497  2B		DEC	HL		+
D498  C0		RET	NZ		.
D499  1A		LD	A,(DE)		.
D49A  77		LD	(HL),A		w
D49B  13		INC	DE		.
D49C  23		INC	HL		#
D49D  1A		LD	A,(DE)		.
D49E  77		LD	(HL),A		w
D49F  1B		DEC	DE		.
D4A0  2B		DEC	HL		+
D4A1  C9		RET			.
		;
D4A2  AF	AD4A2:	XOR	A		.
D4A3  3245CF		LD	(DCF45),A	2E.
D4A6  32EAD9		LD	(DD9EA),A	2..
D4A9  32EBD9		LD	(DD9EB),A	2..
D4AC  CD1ED1		CALL	AD11E		...
D4AF  C0		RET	NZ		.
D4B0  CD69D1		CALL	AD169		.i.
D4B3  E680		AND	080H		..
D4B5  C0		RET	NZ		.
D4B6  0E0F		LD	C,00FH		..
D4B8  CD18D3		CALL	AD318		...
D4BB  CDF5D1		CALL	AD1F5		...
D4BE  C8		RET	Z		.
D4BF  011000		LD	BC,00010H	...
D4C2  CD5ED1		CALL	AD15E		.^.
D4C5  09		ADD	HL,BC		.
D4C6  EB		EX	DE,HL		.
D4C7  2A43CF		LD	HL,(DCF43)	*C.
D4CA  09		ADD	HL,BC		.
D4CB  0E10		LD	C,010H		..
D4CD  3ADDD9	AD4CD:	LD	A,(DD9DD)	:..
D4D0  B7		OR	A		.
D4D1  CAE8D4		JP	Z,AD4E8		...
D4D4  7E		LD	A,(HL)		~
D4D5  B7		OR	A		.
D4D6  1A		LD	A,(DE)		.
D4D7  C2DBD4		JP	NZ,AD4DB	...
D4DA  77		LD	(HL),A		w
D4DB  B7	AD4DB:	OR	A		.
D4DC  C2E1D4		JP	NZ,AD4E1	...
D4DF  7E		LD	A,(HL)		~
D4E0  12		LD	(DE),A		.
D4E1  BE	AD4E1:	CP	(HL)		.
D4E2  C21FD5		JP	NZ,AD51F	...
D4E5  C3FDD4		JP	AD4FD		...
		;
D4E8  CD94D4	AD4E8:	CALL	AD494		...
D4EB  EB		EX	DE,HL		.
D4EC  CD94D4		CALL	AD494		...
D4EF  EB		EX	DE,HL		.
D4F0  1A		LD	A,(DE)		.
D4F1  BE		CP	(HL)		.
D4F2  C21FD5		JP	NZ,AD51F	...
D4F5  13		INC	DE		.
D4F6  23		INC	HL		#
D4F7  1A		LD	A,(DE)		.
D4F8  BE		CP	(HL)		.
D4F9  C21FD5		JP	NZ,AD51F	...
D4FC  0D		DEC	C		.
D4FD  13	AD4FD:	INC	DE		.
D4FE  23		INC	HL		#
D4FF  0D		DEC	C		.
D500  C2CDD4		JP	NZ,AD4CD	...
D503  01ECFF		LD	BC,0FFECH	...
D506  09		ADD	HL,BC		.
D507  EB		EX	DE,HL		.
D508  09		ADD	HL,BC		.
D509  1A		LD	A,(DE)		.
D50A  BE		CP	(HL)		.
D50B  DA17D5		JP	C,AD517		...
D50E  77		LD	(HL),A		w
D50F  010300		LD	BC,00003H	...
D512  09		ADD	HL,BC		.
D513  EB		EX	DE,HL		.
D514  09		ADD	HL,BC		.
D515  7E		LD	A,(HL)		~
D516  12		LD	(DE),A		.
D517  3EFF	AD517:	LD	A,0FFH		>.
D519  32D2D9		LD	(DD9D2),A	2..
D51C  C310D4		JP	AD410		...
		;
D51F  2145CF	AD51F:	LD	HL,DCF45	!E.
D522  35		DEC	(HL)		5
D523  C9		RET			.
		;
D524  CD54D1	AD524:	CALL	AD154		.T.
D527  2A43CF		LD	HL,(DCF43)	*C.
D52A  E5		PUSH	HL		.
D52B  21ACD9		LD	HL,TD9AC	!..
D52E  2243CF		LD	(DCF43),HL	"C.
D531  0E01		LD	C,001H		..
D533  CD18D3		CALL	AD318		...
D536  CDF5D1		CALL	AD1F5		...
D539  E1		POP	HL		.
D53A  2243CF		LD	(DCF43),HL	"C.
D53D  C8		RET	Z		.
D53E  EB		EX	DE,HL		.
D53F  210F00		LD	HL,0000FH	!..
D542  19		ADD	HL,DE		.
D543  0E11		LD	C,011H		..
D545  AF		XOR	A		.
D546  77	AD546:	LD	(HL),A		w
D547  23		INC	HL		#
D548  0D		DEC	C		.
D549  C246D5		JP	NZ,AD546	.F.
D54C  210D00		LD	HL,0000DH	!..
D54F  19		ADD	HL,DE		.
D550  77		LD	(HL),A		w
D551  CD8CD1		CALL	AD18C		...
D554  CDFDD3		CALL	AD3FD		...
D557  C378D1		JP	AD178		.x.
		;
D55A  AF	AD55A:	XOR	A		.
D55B  32D2D9		LD	(DD9D2),A	2..
D55E  CDA2D4		CALL	AD4A2		...
D561  CDF5D1		CALL	AD1F5		...
D564  C8		RET	Z		.
D565  2A43CF		LD	HL,(DCF43)	*C.
D568  010C00		LD	BC,0000CH	...
D56B  09		ADD	HL,BC		.
D56C  7E		LD	A,(HL)		~
D56D  3C		INC	A		<
D56E  E61F		AND	01FH		..
D570  77		LD	(HL),A		w
D571  CA83D5		JP	Z,AD583		...
D574  47		LD	B,A		G
D575  3AC5D9		LD	A,(DD9C5)	:..
D578  A0		AND	B		.
D579  21D2D9		LD	HL,DD9D2	!..
D57C  A6		AND	(HL)		.
D57D  CA8ED5		JP	Z,AD58E		...
D580  C3ACD5		JP	AD5AC		...
		;
D583  010200	AD583:	LD	BC,00002H	...
D586  09		ADD	HL,BC		.
D587  34		INC	(HL)		4
D588  7E		LD	A,(HL)		~
D589  E60F		AND	00FH		..
D58B  CAB6D5		JP	Z,AD5B6		...
D58E  0E0F	AD58E:	LD	C,00FH		..
D590  CD18D3		CALL	AD318		...
D593  CDF5D1		CALL	AD1F5		...
D596  C2ACD5		JP	NZ,AD5AC	...
D599  3AD3D9		LD	A,(DD9D3)	:..
D59C  3C		INC	A		<
D59D  CAB6D5		JP	Z,AD5B6		...
D5A0  CD24D5		CALL	AD524		.$.
D5A3  CDF5D1		CALL	AD1F5		...
D5A6  CAB6D5		JP	Z,AD5B6		...
D5A9  C3AFD5		JP	AD5AF		...
		;
D5AC  CD5AD4	AD5AC:	CALL	AD45A		.Z.
D5AF  CDBBD0	AD5AF:	CALL	AD0BB		...
D5B2  AF		XOR	A		.
D5B3  C301CF		JP	ACF01		...
		;
D5B6  CD05CF	AD5B6:	CALL	ACF05		...
D5B9  C378D1		JP	AD178		.x.
		;
D5BC  3E01	AD5BC:	LD	A,001H		>.
D5BE  32D5D9		LD	(DD9D5),A	2..
D5C1  3EFF	AD5C1:	LD	A,0FFH		>.
D5C3  32D3D9		LD	(DD9D3),A	2..
D5C6  CDBBD0		CALL	AD0BB		...
D5C9  3AE3D9		LD	A,(DD9E3)	:..
D5CC  21E1D9		LD	HL,DD9E1	!..
D5CF  BE		CP	(HL)		.
D5D0  DAE6D5		JP	C,AD5E6		...
D5D3  FE80		CP	080H		..
D5D5  C2FBD5		JP	NZ,AD5FB	...
D5D8  CD5AD5		CALL	AD55A		.Z.
D5DB  AF		XOR	A		.
D5DC  32E3D9		LD	(DD9E3),A	2..
D5DF  3A45CF		LD	A,(DCF45)	:E.
D5E2  B7		OR	A		.
D5E3  C2FBD5		JP	NZ,AD5FB	...
D5E6  CD77D0	AD5E6:	CALL	AD077		.w.
D5E9  CD84D0		CALL	AD084		...
D5EC  CAFBD5		JP	Z,AD5FB		...
D5EF  CD8AD0		CALL	AD08A		...
D5F2  CDD1CF		CALL	ACFD1		...
D5F5  CDB2CF		CALL	ACFB2		...
D5F8  C3D2D0		JP	AD0D2		...
		;
D5FB  C305CF	AD5FB:	JP	ACF05		...
		;
D5FE  3E01	AD5FE:	LD	A,001H		>.
D600  32D5D9		LD	(DD9D5),A	2..
D603  3E00	AD603:	LD	A,000H		>.
D605  32D3D9		LD	(DD9D3),A	2..
D608  CD54D1		CALL	AD154		.T.
D60B  2A43CF		LD	HL,(DCF43)	*C.
D60E  CD47D1		CALL	AD147		.G.
D611  CDBBD0		CALL	AD0BB		...
D614  3AE3D9		LD	A,(DD9E3)	:..
D617  FE80		CP	080H		..
D619  D205CF		JP	NC,ACF05	...
D61C  CD77D0		CALL	AD077		.w.
D61F  CD84D0		CALL	AD084		...
D622  0E00		LD	C,000H		..
D624  C26ED6		JP	NZ,AD66E	.n.
D627  CD3ED0		CALL	AD03E		.>.
D62A  32D7D9		LD	(DD9D7),A	2..
D62D  010000		LD	BC,00000H	...
D630  B7		OR	A		.
D631  CA3BD6		JP	Z,AD63B		.;.
D634  4F		LD	C,A		O
D635  0B		DEC	BC		.
D636  CD5ED0		CALL	AD05E		.^.
D639  44		LD	B,H		D
D63A  4D		LD	C,L		M
D63B  CDBED3	AD63B:	CALL	AD3BE		...
D63E  7D		LD	A,L		}
D63F  B4		OR	H		.
D640  C248D6		JP	NZ,AD648	.H.
D643  3E02		LD	A,002H		>.
D645  C301CF		JP	ACF01		...
		;
D648  22E5D9	AD648:	LD	(DD9E5),HL	"..
D64B  EB		EX	DE,HL		.
D64C  2A43CF		LD	HL,(DCF43)	*C.
D64F  011000		LD	BC,00010H	...
D652  09		ADD	HL,BC		.
D653  3ADDD9		LD	A,(DD9DD)	:..
D656  B7		OR	A		.
D657  3AD7D9		LD	A,(DD9D7)	:..
D65A  CA64D6		JP	Z,AD664		.d.
D65D  CD64D1		CALL	AD164		.d.
D660  73		LD	(HL),E		s
D661  C36CD6		JP	AD66C		.l.
		;
D664  4F	AD664:	LD	C,A		O
D665  0600		LD	B,000H		..
D667  09		ADD	HL,BC		.
D668  09		ADD	HL,BC		.
D669  73		LD	(HL),E		s
D66A  23		INC	HL		#
D66B  72		LD	(HL),D		r
D66C  0E02	AD66C:	LD	C,002H		..
D66E  3A45CF	AD66E:	LD	A,(DCF45)	:E.
D671  B7		OR	A		.
D672  C0		RET	NZ		.
D673  C5		PUSH	BC		.
D674  CD8AD0		CALL	AD08A		...
D677  3AD5D9		LD	A,(DD9D5)	:..
D67A  3D		DEC	A		=
D67B  3D		DEC	A		=
D67C  C2BBD6		JP	NZ,AD6BB	...
D67F  C1		POP	BC		.
D680  C5		PUSH	BC		.
D681  79		LD	A,C		y
D682  3D		DEC	A		=
D683  3D		DEC	A		=
D684  C2BBD6		JP	NZ,AD6BB	...
D687  E5		PUSH	HL		.
D688  2AB9D9		LD	HL,(DD9B9)	*..
D68B  57		LD	D,A		W
D68C  77	AD68C:	LD	(HL),A		w
D68D  23		INC	HL		#
D68E  14		INC	D		.
D68F  F28CD6		JP	P,AD68C		...
D692  CDE0D1		CALL	AD1E0		...
D695  2AE7D9		LD	HL,(DD9E7)	*..
D698  0E02		LD	C,002H		..
D69A  22E5D9	AD69A:	LD	(DD9E5),HL	"..
D69D  C5		PUSH	BC		.
D69E  CDD1CF		CALL	ACFD1		...
D6A1  C1		POP	BC		.
D6A2  CDB8CF		CALL	ACFB8		...
D6A5  2AE5D9		LD	HL,(DD9E5)	*..
D6A8  0E00		LD	C,000H		..
D6AA  3AC4D9		LD	A,(DD9C4)	:..
D6AD  47		LD	B,A		G
D6AE  A5		AND	L		.
D6AF  B8		CP	B		.
D6B0  23		INC	HL		#
D6B1  C29AD6		JP	NZ,AD69A	...
D6B4  E1		POP	HL		.
D6B5  22E5D9		LD	(DD9E5),HL	"..
D6B8  CDDAD1		CALL	AD1DA		...
D6BB  CDD1CF	AD6BB:	CALL	ACFD1		...
D6BE  C1		POP	BC		.
D6BF  C5		PUSH	BC		.
D6C0  CDB8CF		CALL	ACFB8		...
D6C3  C1		POP	BC		.
D6C4  3AE3D9		LD	A,(DD9E3)	:..
D6C7  21E1D9		LD	HL,DD9E1	!..
D6CA  BE		CP	(HL)		.
D6CB  DAD2D6		JP	C,AD6D2		...
D6CE  77		LD	(HL),A		w
D6CF  34		INC	(HL)		4
D6D0  0E02		LD	C,002H		..
D6D2  00	AD6D2:	NOP			.
D6D3  00		NOP			.
D6D4  2100C4		LD	HL,DC400	!..
D6D7  F5		PUSH	AF		.
D6D8  CD69D1		CALL	AD169		.i.
D6DB  E67F		AND	07FH		..
D6DD  77		LD	(HL),A		w
D6DE  F1		POP	AF		.
D6DF  FE7F		CP	07FH		..
D6E1  C200D7		JP	NZ,AD700	...
D6E4  3AD5D9		LD	A,(DD9D5)	:..
D6E7  FE01		CP	001H		..
D6E9  C200D7		JP	NZ,AD700	...
D6EC  CDD2D0		CALL	AD0D2		...
D6EF  CD5AD5		CALL	AD55A		.Z.
D6F2  2145CF		LD	HL,DCF45	!E.
D6F5  7E		LD	A,(HL)		~
D6F6  B7		OR	A		.
D6F7  C2FED6		JP	NZ,AD6FE	...
D6FA  3D		DEC	A		=
D6FB  32E3D9		LD	(DD9E3),A	2..
D6FE  3600	AD6FE:	LD	(HL),000H	6.
D700  C3D2D0	AD700:	JP	AD0D2		...
		;
D703  AF	AD703:	XOR	A		.
D704  32D5D9		LD	(DD9D5),A	2..
D707  C5	AD707:	PUSH	BC		.
D708  2A43CF		LD	HL,(DCF43)	*C.
D70B  EB		EX	DE,HL		.
D70C  212100		LD	HL,00021H	!!.
D70F  19		ADD	HL,DE		.
D710  7E		LD	A,(HL)		~
D711  E67F		AND	07FH		..
D713  F5		PUSH	AF		.
D714  7E		LD	A,(HL)		~
D715  17		RLA			.
D716  23		INC	HL		#
D717  7E		LD	A,(HL)		~
D718  17		RLA			.
D719  E61F		AND	01FH		..
D71B  4F		LD	C,A		O
D71C  7E		LD	A,(HL)		~
D71D  1F		RRA			.
D71E  1F		RRA			.
D71F  1F		RRA			.
D720  1F		RRA			.
D721  E60F		AND	00FH		..
D723  47		LD	B,A		G
D724  F1		POP	AF		.
D725  23		INC	HL		#
D726  6E		LD	L,(HL)		n
D727  2C		INC	L		,
D728  2D		DEC	L		-
D729  2E06		LD	L,006H		..
D72B  C28BD7		JP	NZ,AD78B	...
D72E  212000		LD	HL,00020H	! .
D731  19		ADD	HL,DE		.
D732  77		LD	(HL),A		w
D733  210C00		LD	HL,0000CH	!..
D736  19		ADD	HL,DE		.
D737  79		LD	A,C		y
D738  96		SUB	(HL)		.
D739  C247D7		JP	NZ,AD747	.G.
D73C  210E00		LD	HL,0000EH	!..
D73F  19		ADD	HL,DE		.
D740  78		LD	A,B		x
D741  96		SUB	(HL)		.
D742  E67F		AND	07FH		..
D744  CA7FD7		JP	Z,AD77F		...
D747  C5	AD747:	PUSH	BC		.
D748  D5		PUSH	DE		.
D749  CDA2D4		CALL	AD4A2		...
D74C  D1		POP	DE		.
D74D  C1		POP	BC		.
D74E  2E03		LD	L,003H		..
D750  3A45CF		LD	A,(DCF45)	:E.
D753  3C		INC	A		<
D754  CA84D7		JP	Z,AD784		...
D757  210C00		LD	HL,0000CH	!..
D75A  19		ADD	HL,DE		.
D75B  71		LD	(HL),C		q
D75C  210E00		LD	HL,0000EH	!..
D75F  19		ADD	HL,DE		.
D760  70		LD	(HL),B		p
D761  CD51D4		CALL	AD451		.Q.
D764  3A45CF		LD	A,(DCF45)	:E.
D767  3C		INC	A		<
D768  C27FD7		JP	NZ,AD77F	...
D76B  C1		POP	BC		.
D76C  C5		PUSH	BC		.
D76D  2E04		LD	L,004H		..
D76F  0C		INC	C		.
D770  CA84D7		JP	Z,AD784		...
D773  CD24D5		CALL	AD524		.$.
D776  2E05		LD	L,005H		..
D778  3A45CF		LD	A,(DCF45)	:E.
D77B  3C		INC	A		<
D77C  CA84D7		JP	Z,AD784		...
D77F  C1	AD77F:	POP	BC		.
D780  AF		XOR	A		.
D781  C301CF		JP	ACF01		...
		;
D784  E5	AD784:	PUSH	HL		.
D785  CD69D1		CALL	AD169		.i.
D788  36C0		LD	(HL),0C0H	6.
D78A  E1		POP	HL		.
D78B  C1	AD78B:	POP	BC		.
D78C  7D		LD	A,L		}
D78D  3245CF		LD	(DCF45),A	2E.
D790  C378D1		JP	AD178		.x.
		;
D793  0EFF	AD793:	LD	C,0FFH		..
D795  CD03D7		CALL	AD703		...
D798  CCC1D5		CALL	Z,AD5C1		...
D79B  C9		RET			.
		;
D79C  0E00	AD79C:	LD	C,000H		..
D79E  CD03D7		CALL	AD703		...
D7A1  CC03D6		CALL	Z,AD603		...
D7A4  C9		RET			.
		;
D7A5  EB	AD7A5:	EX	DE,HL		.
D7A6  19		ADD	HL,DE		.
D7A7  4E		LD	C,(HL)		N
D7A8  0600		LD	B,000H		..
D7AA  210C00		LD	HL,0000CH	!..
D7AD  19		ADD	HL,DE		.
D7AE  7E		LD	A,(HL)		~
D7AF  0F		RRCA			.
D7B0  E680		AND	080H		..
D7B2  81		ADD	A,C		.
D7B3  4F		LD	C,A		O
D7B4  3E00		LD	A,000H		>.
D7B6  88		ADC	A,B		.
D7B7  47		LD	B,A		G
D7B8  7E		LD	A,(HL)		~
D7B9  0F		RRCA			.
D7BA  E60F		AND	00FH		..
D7BC  80		ADD	A,B		.
D7BD  47		LD	B,A		G
D7BE  210E00		LD	HL,0000EH	!..
D7C1  19		ADD	HL,DE		.
D7C2  7E		LD	A,(HL)		~
D7C3  87		ADD	A,A		.
D7C4  87		ADD	A,A		.
D7C5  87		ADD	A,A		.
D7C6  87		ADD	A,A		.
D7C7  F5		PUSH	AF		.
D7C8  80		ADD	A,B		.
D7C9  47		LD	B,A		G
D7CA  F5		PUSH	AF		.
D7CB  E1		POP	HL		.
D7CC  7D		LD	A,L		}
D7CD  E1		POP	HL		.
D7CE  B5		OR	L		.
D7CF  E601		AND	001H		..
D7D1  C9		RET			.
		;
D7D2  0E0C	AD7D2:	LD	C,00CH		..
D7D4  CD18D3		CALL	AD318		...
D7D7  2A43CF		LD	HL,(DCF43)	*C.
D7DA  112100		LD	DE,00021H	.!.
D7DD  19		ADD	HL,DE		.
D7DE  E5		PUSH	HL		.
D7DF  72		LD	(HL),D		r
D7E0  23		INC	HL		#
D7E1  72		LD	(HL),D		r
D7E2  23		INC	HL		#
D7E3  72		LD	(HL),D		r
D7E4  CDF5D1	AD7E4:	CALL	AD1F5		...
D7E7  CA0CD8		JP	Z,AD80C		...
D7EA  CD5ED1		CALL	AD15E		.^.
D7ED  110F00		LD	DE,0000FH	...
D7F0  CDA5D7		CALL	AD7A5		...
D7F3  E1		POP	HL		.
D7F4  E5		PUSH	HL		.
D7F5  5F		LD	E,A		_
D7F6  79		LD	A,C		y
D7F7  96		SUB	(HL)		.
D7F8  23		INC	HL		#
D7F9  78		LD	A,B		x
D7FA  9E		SBC	A,(HL)		.
D7FB  23		INC	HL		#
D7FC  7B		LD	A,E		{
D7FD  9E		SBC	A,(HL)		.
D7FE  DA06D8		JP	C,AD806		...
D801  73		LD	(HL),E		s
D802  2B		DEC	HL		+
D803  70		LD	(HL),B		p
D804  2B		DEC	HL		+
D805  71		LD	(HL),C		q
D806  CD2DD3	AD806:	CALL	AD32D		.-.
D809  C3E4D7		JP	AD7E4		...
		;
D80C  E1	AD80C:	POP	HL		.
D80D  C9		RET			.
		;
		; >> NO EXECUTION PATH TO HERE <<
D80E  2A43CF		LD	HL,(DCF43)	*C.
D811  112000		LD	DE,00020H	. .
D814  CDA5D7		CALL	AD7A5		...
D817  212100		LD	HL,00021H	!!.
D81A  19		ADD	HL,DE		.
D81B  71		LD	(HL),C		q
D81C  23		INC	HL		#
D81D  70		LD	(HL),B		p
D81E  23		INC	HL		#
D81F  77		LD	(HL),A		w
D820  C9		RET			.
		;
D821  2AAFD9	AD821:	LD	HL,(DD9AF)	*..
D824  3A42CF		LD	A,(DCF42)	:B.
D827  4F		LD	C,A		O
D828  CDEAD0		CALL	AD0EA		...
D82B  E5		PUSH	HL		.
D82C  EB		EX	DE,HL		.
D82D  CD59CF		CALL	ACF59		.Y.
D830  E1		POP	HL		.
D831  CC47CF		CALL	Z,ACF47		.G.
D834  7D		LD	A,L		}
D835  1F		RRA			.
D836  D8		RET	C		.
D837  2AAFD9		LD	HL,(DD9AF)	*..
D83A  4D		LD	C,L		M
D83B  44		LD	B,H		D
D83C  CD0BD1		CALL	AD10B		...
D83F  22AFD9		LD	(DD9AF),HL	"..
D842  C3A3D2		JP	AD2A3		...
		;
D845  3AD6D9	AD845:	LD	A,(DD9D6)	:..
D848  2142CF		LD	HL,DCF42	!B.
D84B  BE		CP	(HL)		.
D84C  C8		RET	Z		.
D84D  77		LD	(HL),A		w
D84E  C321D8		JP	AD821		.!.
		;
D851  3EFF	AD851:	LD	A,0FFH		>.
D853  32DED9		LD	(DD9DE),A	2..
D856  2A43CF		LD	HL,(DCF43)	*C.
D859  7E		LD	A,(HL)		~
D85A  E61F		AND	01FH		..
D85C  3D		DEC	A		=
D85D  32D6D9		LD	(DD9D6),A	2..
D860  FE1E		CP	01EH		..
D862  D275D8		JP	NC,AD875	.u.
D865  3A42CF		LD	A,(DCF42)	:B.
D868  32DFD9		LD	(DD9DF),A	2..
D86B  7E		LD	A,(HL)		~
D86C  32E0D9		LD	(DD9E0),A	2..
D86F  E6E0		AND	0E0H		..
D871  77		LD	(HL),A		w
D872  CD45D8		CALL	AD845		.E.
D875  3A41CF	AD875:	LD	A,(DCF41)	:A.
D878  2A43CF		LD	HL,(DCF43)	*C.
D87B  B6		OR	(HL)		.
D87C  77		LD	(HL),A		w
D87D  C9		RET			.
		;
		; >> NO EXECUTION PATH TO HERE <<
D87E  3E22		LD	A,022H		>"
D880  C301CF		JP	ACF01		...
		;
		; >> NO EXECUTION PATH TO HERE <<
D883  210000		LD	HL,00000H	!..
D886  22ADD9		LD	(DD9AD),HL	"..
D889  22AFD9		LD	(DD9AF),HL	"..
D88C  AF		XOR	A		.
D88D  3242CF		LD	(DCF42),A	2B.
D890  218000		LD	HL,00080H	!..
D893  22B1D9		LD	(DD9B1),HL	"..
D896  CDDAD1		CALL	AD1DA		...
D899  C321D8		JP	AD821		.!.
		;
		; >> NO EXECUTION PATH TO HERE <<
D89C  CD72D1		CALL	AD172		.r.
D89F  CD51D8		CALL	AD851		.Q.
D8A2  C351D4		JP	AD451		.Q.
		;
		; >> NO EXECUTION PATH TO HERE <<
D8A5  CD51D8		CALL	AD851		.Q.
D8A8  C3A2D4		JP	AD4A2		...
		;
		; >> NO EXECUTION PATH TO HERE <<
D8AB  0E00		LD	C,000H		..
D8AD  EB		EX	DE,HL		.
D8AE  7E		LD	A,(HL)		~
D8AF  FE3F		CP	03FH		.?
D8B1  CAC2D8		JP	Z,AD8C2		...
D8B4  CDA6D0		CALL	AD0A6		...
D8B7  7E		LD	A,(HL)		~
D8B8  FE3F		CP	03FH		.?
D8BA  C472D1		CALL	NZ,AD172	.r.
D8BD  CD51D8		CALL	AD851		.Q.
D8C0  0E0F		LD	C,00FH		..
D8C2  CD18D3	AD8C2:	CALL	AD318		...
D8C5  C3E9D1		JP	AD1E9		...
		;
		; >> NO EXECUTION PATH TO HERE <<
D8C8  2AD9D9		LD	HL,(DD9D9)	*..
D8CB  2243CF		LD	(DCF43),HL	"C.
D8CE  CD51D8		CALL	AD851		.Q.
D8D1  CD2DD3		CALL	AD32D		.-.
D8D4  C3E9D1		JP	AD1E9		...
		;
		; >> NO EXECUTION PATH TO HERE <<
D8D7  CD51D8		CALL	AD851		.Q.
D8DA  CD9CD3		CALL	AD39C		...
D8DD  C301D3		JP	AD301		...
		;
		; >> NO EXECUTION PATH TO HERE <<
D8E0  CD51D8		CALL	AD851		.Q.
D8E3  C3BCD5		JP	AD5BC		...
		;
		; >> NO EXECUTION PATH TO HERE <<
D8E6  CD51D8		CALL	AD851		.Q.
D8E9  C3FED5		JP	AD5FE		...
		;
		; >> NO EXECUTION PATH TO HERE <<
D8EC  CD72D1		CALL	AD172		.r.
D8EF  CD51D8		CALL	AD851		.Q.
D8F2  C324D5		JP	AD524		.$.
		;
		; >> NO EXECUTION PATH TO HERE <<
D8F5  CD51D8		CALL	AD851		.Q.
D8F8  CD16D4		CALL	AD416		...
D8FB  C301D3		JP	AD301		...
		;
		; >> NO EXECUTION PATH TO HERE <<
D8FE  2AAFD9		LD	HL,(DD9AF)	*..
D901  C329D9		JP	AD929		.).
		;
		; >> NO EXECUTION PATH TO HERE <<
D904  3A42CF		LD	A,(DCF42)	:B.
D907  C301CF		JP	ACF01		...
		;
		; >> NO EXECUTION PATH TO HERE <<
D90A  EB		EX	DE,HL		.
D90B  22B1D9		LD	(DD9B1),HL	"..
D90E  C3DAD1		JP	AD1DA		...
		;
		; >> NO EXECUTION PATH TO HERE <<
D911  2ABFD9		LD	HL,(DD9BF)	*..
D914  C329D9		JP	AD929		.).
		;
		; >> NO EXECUTION PATH TO HERE <<
D917  2AADD9		LD	HL,(DD9AD)	*..
D91A  C329D9		JP	AD929		.).
		;
		; >> NO EXECUTION PATH TO HERE <<
D91D  CD51D8		CALL	AD851		.Q.
D920  CD3BD4		CALL	AD43B		.;.
D923  C301D3		JP	AD301		...
		;
		; >> NO EXECUTION PATH TO HERE <<
D926  2ABBD9		LD	HL,(DD9BB)	*..
D929  2245CF	AD929:	LD	(DCF45),HL	"E.
D92C  C9		RET			.
		;
		; >> NO EXECUTION PATH TO HERE <<
D92D  3AD6D9		LD	A,(DD9D6)	:..
D930  FEFF		CP	0FFH		..
D932  C23BD9		JP	NZ,AD93B	.;.
D935  3A41CF		LD	A,(DCF41)	:A.
D938  C301CF		JP	ACF01		...
		;
D93B  E61F	AD93B:	AND	01FH		..
D93D  3241CF		LD	(DCF41),A	2A.
D940  C9		RET			.
		;
		; >> NO EXECUTION PATH TO HERE <<
D941  CD51D8		CALL	AD851		.Q.
D944  C393D7		JP	AD793		...
		;
		; >> NO EXECUTION PATH TO HERE <<
D947  CD51D8		CALL	AD851		.Q.
D94A  C39CD7		JP	AD79C		...
		;
		; >> NO EXECUTION PATH TO HERE <<
D94D  CD51D8		CALL	AD851		.Q.
D950  C3D2D7		JP	AD7D2		...
		;
		; >> NO EXECUTION PATH TO HERE <<
D953  2A43CF		LD	HL,(DCF43)	*C.
D956  7D		LD	A,L		}
D957  2F		CPL			/
D958  5F		LD	E,A		_
D959  7C		LD	A,H		|
D95A  2F		CPL			/
D95B  2AAFD9		LD	HL,(DD9AF)	*..
D95E  A4		AND	H		.
D95F  57		LD	D,A		W
D960  7D		LD	A,L		}
D961  A3		AND	E		.
D962  5F		LD	E,A		_
D963  2AADD9		LD	HL,(DD9AD)	*..
D966  EB		EX	DE,HL		.
D967  22AFD9		LD	(DD9AF),HL	"..
D96A  7D		LD	A,L		}
D96B  A3		AND	E		.
D96C  6F		LD	L,A		o
D96D  7C		LD	A,H		|
D96E  A2		AND	D		.
D96F  67		LD	H,A		g
D970  22ADD9		LD	(DD9AD),HL	"..
D973  C9		RET			.
		;
D974  3ADED9	AD974:	LD	A,(DD9DE)	:..
D977  B7		OR	A		.
D978  CA91D9		JP	Z,AD991		...
D97B  2A43CF		LD	HL,(DCF43)	*C.
D97E  3600		LD	(HL),000H	6.
D980  3AE0D9		LD	A,(DD9E0)	:..
D983  B7		OR	A		.
D984  CA91D9		JP	Z,AD991		...
D987  77		LD	(HL),A		w
D988  3ADFD9		LD	A,(DD9DF)	:..
D98B  32D6D9		LD	(DD9D6),A	2..
D98E  CD45D8		CALL	AD845		.E.
D991  2A0FCF	AD991:	LD	HL,(DCF0F)	*..
D994  F9		LD	SP,HL		.
D995  2A45CF		LD	HL,(DCF45)	*E.
D998  7D		LD	A,L		}
D999  44		LD	B,H		D
D99A  C9		RET			.
		;
		; >> NO EXECUTION PATH TO HERE <<
D99B  CD51D8		CALL	AD851		.Q.
D99E  3E02		LD	A,002H		>.
D9A0  32D5D9		LD	(DD9D5),A	2..
D9A3  0E00		LD	C,000H		..
D9A5  CD07D7		CALL	AD707		...
D9A8  CC03D6		CALL	Z,AD603		...
D9AB  C9		RET			.
		;
		; >> NO EXECUTION PATH TO HERE <<
D9AC  E5	TD9AC:	PUSH	HL		.
D9AD  00	DD9AD:	NOP			.
D9AE  00		NOP			.
D9AF  05	DD9AF:	DEC	B		.
D9B0  00		NOP			.
D9B1  80	DD9B1:	ADD	A,B		.
D9B2  00		NOP			.
D9B3  6C	DD9B3:	LD	L,H		l
D9B4  DA6EDA		JP	C,XDA6E		.n.
D9B7  70	DD9B7:	LD	(HL),B		p
D9B8  DA50F4		JP	C,XF450		.P.
D9BB  8B	DD9BB:	ADC	A,E		.
D9BC  DAABF5		JP	C,XF5AB		...
D9BF  72	DD9BF:	LD	(HL),D		r
D9C0  F5		PUSH	AF		.
D9C1  010004	DD9C1:	LD	BC,00400H	...
D9C4  0F	DD9C4:	RRCA			.
D9C5  00	DD9C5:	NOP			.
D9C6  94	DD9C6:	SUB	H		.
D9C7  00		NOP			.
D9C8  7F	DD9C8:	LD	A,A		.
D9C9  00		NOP			.
D9CA  C0	DD9CA:	RET	NZ		.
D9CB  00		NOP			.
...
D9D5  00	DD9D5:	NOP			.
D9D6  0600	DD9D6:	LD	B,000H		..
D9D8  00	DD9D8:	NOP			.
...
D9DC  00		NOP			.
D9DD  FF	DD9DD:	RST	038H		.
D9DE  00	DD9DE:	NOP			.
...
D9E4  00		NOP			.
D9E5  1F	DD9E5:	RRA			.
D9E6  00		NOP			.
D9E7  00	DD9E7:	NOP			.
D9E8  00		NOP			.
D9E9  60	DD9E9:	LD	H,B		`
D9EA  FF	DD9EA:	RST	038H		.
D9EB  FF	DD9EB:	RST	038H		.
D9EC  1F	DD9EC:	RRA			.
D9ED  00		NOP			.
...
D9FE  00		NOP			.
			END

LABELS ON FILE CCP.LBL
